 unpack200

 Timestamp is b1d1b15f (reproducible build file hash)

 Preferred load address is 0000000140000000

 Start         Length     Name                   Class
 0001:00000000 00014940H .text$mn                CODE
 0001:00014940 00000036H .text$mn$00             CODE
 0001:00014976 00000036H .text$x                 CODE
 0002:00000000 000002c0H .idata$5                DATA
 0002:000002c0 00000038H .00cfg                  DATA
 0002:000002f8 00000008H .CRT$XCA                DATA
 0002:00000300 00000008H .CRT$XCAA               DATA
 0002:00000308 00000008H .CRT$XCZ                DATA
 0002:00000310 00000008H .CRT$XIA                DATA
 0002:00000318 00000008H .CRT$XIAA               DATA
 0002:00000320 00000008H .CRT$XIAC               DATA
 0002:00000328 00000008H .CRT$XIZ                DATA
 0002:00000330 00000008H .CRT$XPA                DATA
 0002:00000338 00000008H .CRT$XPZ                DATA
 0002:00000340 00000008H .CRT$XTA                DATA
 0002:00000348 00000008H .CRT$XTZ                DATA
 0002:00000350 00000000H .gehcont$y              DATA
 0002:00000350 00000000H .gfids$y                DATA
 0002:00000350 00007f30H .rdata                  DATA
 0002:00008280 00000000H .rdata$CastGuardVftablesA DATA
 0002:00008280 00000000H .rdata$CastGuardVftablesC DATA
 0002:00008280 00000060H .rdata$voltmd           DATA
 0002:000082e0 000002f8H .rdata$zzzdbg           DATA
 0002:000085d8 00000008H .rtc$IAA                DATA
 0002:000085e0 00000008H .rtc$IZZ                DATA
 0002:000085e8 00000008H .rtc$TAA                DATA
 0002:000085f0 00000008H .rtc$TZZ                DATA
 0002:000085f8 00000808H .xdata                  DATA
 0002:00008e00 00000048H .edata                  DATA
 0002:00008e48 00000104H .idata$2                DATA
 0002:00008f4c 00000014H .idata$3                DATA
 0002:00008f60 000002c0H .idata$4                DATA
 0002:00009220 00000662H .idata$6                DATA
 0003:00000000 00000bb0H .data                   DATA
 0003:00000bb0 00000a20H .bss                    DATA
 0004:00000000 00000960H .pdata                  DATA
 0005:00000000 00000060H .rsrc$01                DATA
 0005:00000060 00000318H .rsrc$02                DATA

  Address         Publics by Value              Rva+Base               Lib:Object

 0000:00000000       __AbsoluteZero             0000000000000000     <absolute>
 0000:00000000       ___safe_se_handler_count   0000000000000000     <absolute>
 0000:00000000       ___safe_se_handler_table   0000000000000000     <absolute>
 0000:00000000       __arm64x_extra_rfe_table   0000000000000000     <absolute>
 0000:00000000       __arm64x_extra_rfe_table_size 0000000000000000     <absolute>
 0000:00000000       __arm64x_native_entrypoint 0000000000000000     <absolute>
 0000:00000000       __arm64x_redirection_metadata 0000000000000000     <absolute>
 0000:00000000       __arm64x_redirection_metadata_count 0000000000000000     <absolute>
 0000:00000000       __dynamic_value_reloc_table 0000000000000000     <absolute>
 0000:00000000       __enclave_config           0000000000000000     <absolute>
 0000:00000000       __guard_check_icall_a64n_fptr 0000000000000000     <absolute>
 0000:00000000       __guard_eh_cont_count      0000000000000000     <absolute>
 0000:00000000       __guard_eh_cont_table      0000000000000000     <absolute>
 0000:00000000       __guard_fids_count         0000000000000000     <absolute>
 0000:00000000       __guard_fids_table         0000000000000000     <absolute>
 0000:00000000       __guard_iat_count          0000000000000000     <absolute>
 0000:00000000       __guard_iat_table          0000000000000000     <absolute>
 0000:00000000       __guard_longjmp_count      0000000000000000     <absolute>
 0000:00000000       __guard_longjmp_table      0000000000000000     <absolute>
 0000:00000000       __hybrid_auxiliary_delayload_iat 0000000000000000     <absolute>
 0000:00000000       __hybrid_auxiliary_delayload_iat_copy 0000000000000000     <absolute>
 0000:00000000       __hybrid_auxiliary_iat     0000000000000000     <absolute>
 0000:00000000       __hybrid_auxiliary_iat_copy 0000000000000000     <absolute>
 0000:00000000       __hybrid_code_map          0000000000000000     <absolute>
 0000:00000000       __hybrid_code_map_count    0000000000000000     <absolute>
 0000:00000000       __hybrid_image_info_bitfield 0000000000000000     <absolute>
 0000:00000000       __x64_code_ranges_to_entry_points 0000000000000000     <absolute>
 0000:00000000       __x64_code_ranges_to_entry_points_count 0000000000000000     <absolute>
 0000:00000100       __guard_flags              0000000000000100     <absolute>
 0000:00000000       __ImageBase                0000000140000000     <linker-defined>
 0001:00000dd0       deflate                    0000000140001dd0 f   deflate.obj
 0001:0000179c       deflateEnd                 000000014000279c f   deflate.obj
 0001:00001850       deflateInit2_              0000000140002850 f   deflate.obj
 0001:00001ad0       deflateReset               0000000140002ad0 f   deflate.obj
 0001:00001b00       deflateResetKeep           0000000140002b00 f   deflate.obj
 0001:000026d4       inflate_fast               00000001400036d4 f   inffast.obj
 0001:00002b14       inflate                    0000000140003b14 f   inflate.obj
 0001:000040f0       inflateEnd                 00000001400050f0 f   inflate.obj
 0001:00004148       inflateInit2_              0000000140005148 f   inflate.obj
 0001:00004224       inflateReset               0000000140005224 f   inflate.obj
 0001:00004250       inflateReset2              0000000140005250 f   inflate.obj
 0001:000042e8       inflateResetKeep           00000001400052e8 f   inflate.obj
 0001:000044ac       inflate_table              00000001400054ac f   inftrees.obj
 0001:00004944       _tr_align                  0000000140005944 f   trees.obj
 0001:00004a28       _tr_flush_bits             0000000140005a28 f   trees.obj
 0001:00004a30       _tr_flush_block            0000000140005a30 f   trees.obj
 0001:00004d54       _tr_init                   0000000140005d54 f   trees.obj
 0001:00004dbc       _tr_stored_block           0000000140005dbc f   trees.obj
 0001:000062cc       adler32                    00000001400072cc f   zadler32.obj
 0001:000062d4       adler32_z                  00000001400072d4 f   zadler32.obj
 0001:000065bc       crc32                      00000001400075bc f   zcrc32.obj
 0001:000065c4       crc32_z                    00000001400075c4 f   zcrc32.obj
 0001:000068d4       zcalloc                    00000001400078d4 f   zutil.obj
 0001:000068e4       zcfree                     00000001400078e4 f   zutil.obj
 0001:000068f0       ?getIntCount@band@@QEAAHH@Z 00000001400078f0 f   bands.obj
 0001:000069f4       ?getIntTotal@band@@QEAAHXZ 00000001400079f4 f   bands.obj
 0001:00006aa8       ?getLong@band@@QEAA_JAEAU1@_N@Z 0000000140007aa8 f   bands.obj
 0001:00006af4       ?getRefCommon@band@@QEAAPEAUentry@@PEAUcpindex@@_N@Z 0000000140007af4 f   bands.obj
 0001:00006b98       ?initIndexes@band@@SAXPEAUunpacker@@@Z 0000000140007b98 f   bands.obj
 0001:00006bec       ?makeBands@band@@SAPEAU1@PEAUunpacker@@@Z 0000000140007bec f   bands.obj
 0001:00006ca0       ?readData@band@@QEAAXH@Z   0000000140007ca0 f   bands.obj
 0001:00006ea8       ?setIndex@band@@QEAAXPEAUcpindex@@@Z 0000000140007ea8 f   bands.obj
 0001:00006eb0       ?setIndexByTag@band@@QEAAXC@Z 0000000140007eb0 f   bands.obj
 0001:00006ee4       ?compareTo@bytes@@QEAAHAEAU1@@Z 0000000140007ee4 f   bytes.obj
 0001:00006f34       ?copyFrom@bytes@@QEAAXPEBX_K1@Z 0000000140007f34 f   bytes.obj
 0001:00006f40       ?ensureSize@fillbytes@@QEAAX_K@Z 0000000140007f40 f   bytes.obj
 0001:00006f70       ?free@bytes@@QEAAXXZ       0000000140007f70 f   bytes.obj
 0001:00006fa4       ?freeAll@ptrlist@@QEAAXXZ  0000000140007fa4 f   bytes.obj
 0001:00007008       ?grow@fillbytes@@QEAAPEAC_K@Z 0000000140008008 f   bytes.obj
 0001:000070d8       ?indexOf@ptrlist@@QEAAHPEBX@Z 00000001400080d8 f   bytes.obj
 0001:00007108       ?malloc@bytes@@QEAAX_K@Z   0000000140008108 f   bytes.obj
 0001:0000716c       ?realloc@bytes@@QEAAX_K@Z  000000014000816c f   bytes.obj
 0001:00007224       ?saveFrom@bytes@@QEAAXPEBX_K@Z 0000000140008224 f   bytes.obj
 0001:0000726c       ?writeTo@bytes@@QEAAPEACPEAC@Z 000000014000826c f   bytes.obj
 0001:000072a0       ?findByIndex@coding@@SAPEAU1@H@Z 00000001400082a0 f   coding.obj
 0001:000072c4       ?findBySpec@coding@@SAPEAU1@H@Z 00000001400082c4 f   coding.obj
 0001:0000733c       ?findBySpec@coding@@SAPEAU1@HHHH@Z 000000014000833c f   coding.obj
 0001:00007374       ?getInt@value_stream@@QEAAHXZ 0000000140008374 f   coding.obj
 0001:000076d8       ?init@coding@@QEAAPEAU1@XZ 00000001400086d8 f   coding.obj
 0001:00007898       ?init@coding_method@@QEAAXAEAPEACPEAC0HPEAUcoding@@HPEAUintlist@@@Z 0000000140008898 f   coding.obj
 0001:00007ff4       ?init@value_stream@@QEAAXPEAC0PEAUcoding@@@Z 0000000140008ff4 f   coding.obj
 0001:00008010       ?parse@coding@@SAIAEAPEACHH@Z 0000000140009010 f   coding.obj
 0001:00008090       ?parseMultiple@coding@@SAXAEAPEACHPEACHH@Z 0000000140009090 f   coding.obj
 0001:00008120       ?parse_lgH@coding@@SAIAEAPEACHHH@Z 0000000140009120 f   coding.obj
 0001:000081a0       ?reset@coding_method@@QEAAXPEAUvalue_stream@@@Z 00000001400091a0 f   coding.obj
 0001:000081f0       ?setCoding@value_stream@@QEAAXPEAUcoding@@@Z 00000001400091f0 f   coding.obj
 0001:00008300       ?sumInUnsignedRange@coding@@QEAAHHH@Z 0000000140009300 f   coding.obj
 0001:00008334       ?current@unpacker@@SAPEAU1@XZ 0000000140009334 f   main.obj
 0001:00008458       ?run@unpacker@@SAHHPEAPEAD@Z 0000000140009458 f   main.obj
 0001:00008cf8       __local_stdio_printf_options 0000000140009cf8 f i main.obj
 0001:00008d00       fprintf                    0000000140009d00 f i main.obj
 0001:00008d44       main                       0000000140009d44 f   main.obj
 0001:00008d4c       sprintf                    0000000140009d4c f i main.obj
 0001:00008da4       ?abort@attr_definitions@unpacker@@QEAAXPEBD@Z 0000000140009da4 f i unpack.obj
 0001:00008db4       ?abort@cpool@@QEAAXPEBD@Z  0000000140009db4 f i unpack.obj
 0001:00008dc8       ?abort@unpacker@@QEAAXPEBD@Z 0000000140009dc8 f   unpack.obj
 0001:00008e04       ?buildBands@attr_definitions@unpacker@@QEAAPEAPEAUband@@PEAUlayout_definition@2@@Z 0000000140009e04 f   unpack.obj
 0001:00008f7c       ?calloc_heap@unpacker@@QEAAPEAX_K0_N1@Z 0000000140009f7c f   unpack.obj
 0001:0000908c       ?checkLegacy@unpacker@@QEAAXPEBD@Z 000000014000a08c f   unpack.obj
 0001:000090fc       ?check_options@unpacker@@QEAAXXZ 000000014000a0fc f   unpack.obj
 0001:00009144       ?close_output@unpacker@@QEAAPEAUfillbytes@@PEAU2@@Z 000000014000a144 f   unpack.obj
 0001:0000925c       ?computeOutputIndexes@cpool@@QEAAXXZ 000000014000a25c f   unpack.obj
 0001:000092e0       ?defineLayout@attr_definitions@unpacker@@QEAAPEAUlayout_definition@2@HPEBD0@Z 000000014000a2e0 f   unpack.obj
 0001:00009400       ?dump_options@unpacker@@QEAAXXZ 000000014000a400 f   unpack.obj
 0001:00009490       ?ensureClass@cpool@@QEAAPEAUentry@@AEAUbytes@@@Z 000000014000a490 f   unpack.obj
 0001:00009564       ?ensureUtf8@cpool@@QEAAPEAUentry@@AEAUbytes@@@Z 000000014000a564 f   unpack.obj
 0001:0000960c       ?ensure_input@unpacker@@QEAA_N_J@Z 000000014000a60c f   unpack.obj
 0001:00009718       ?ensure_put_space@unpacker@@QEAAX_K@Z 000000014000a718 f   unpack.obj
 0001:00009784       ?expandSignatures@cpool@@QEAAXXZ 000000014000a784 f   unpack.obj
 0001:000099a8       ?finish@unpacker@@QEAAXXZ  000000014000a9a8 f   unpack.obj
 0001:00009aa8       ?free@attr_definitions@unpacker@@QEAAXXZ 000000014000aaa8 f i unpack.obj
 0001:00009b44       ?free@unpacker@@QEAAXXZ    000000014000ab44 f   unpack.obj
 0001:00009d94       ?get@cpindex@@QEAAPEAUentry@@I@Z 000000014000ad94 f   unpack.obj
 0001:00009db8       ?getKQIndex@cpool@@QEAAPEAUcpindex@@XZ 000000014000adb8 f   unpack.obj
 0001:00009e48       ?get_abort_message@unpacker@@QEAAPEBDXZ 000000014000ae48 f   unpack.obj
 0001:00009e50       ?get_code_header@unpacker@@QEAAXAEAH000@Z 000000014000ae50 f   unpack.obj
 0001:00009f20       ?get_next_file@unpacker@@QEAAPEAUfile@1@XZ 000000014000af20 f   unpack.obj
 0001:0000a2b0       ?get_option@unpacker@@QEAAPEBDPEBD@Z 000000014000b2b0 f   unpack.obj
 0001:0000a434       ?hashTabRef@cpool@@QEAAAEAPEAUentry@@CAEAUbytes@@@Z 000000014000b434 f   unpack.obj
 0001:0000a514       ?init@cpool@@QEAAXPEAUunpacker@@QEAH@Z 000000014000b514 f   unpack.obj
 0001:0000a6f0       ?init@unpacker@@QEAAXP6A_JPEAU1@PEAX_J2@Z@Z 000000014000b6f0 f   unpack.obj
 0001:0000a79c       ?initGroupIndexes@cpool@@QEAAXXZ 000000014000b79c f   unpack.obj
 0001:0000a8c8       ?initMemberIndexes@cpool@@QEAAXXZ 000000014000b8c8 f   unpack.obj
 0001:0000abc4       ?parseIntLayout@attr_definitions@unpacker@@QEAAPEBDPEBDAEAPEAUband@@C_N@Z 000000014000bbc4 f   unpack.obj
 0001:0000acf4       ?parseLayout@attr_definitions@unpacker@@QEAAPEBDPEBDAEAPEAPEAUband@@H@Z 000000014000bcf4 f   unpack.obj
 0001:0000b488       ?parseNumeral@attr_definitions@unpacker@@QEAAPEBDPEBDAEAH@Z 000000014000c488 f   unpack.obj
 0001:0000b544       ?popBody@attr_definitions@unpacker@@QEAAPEAPEAUband@@H@Z 000000014000c544 f   unpack.obj
 0001:0000b604       ?put_label@unpacker@@QEAAXHH@Z 000000014000c604 f   unpack.obj
 0001:0000b678       ?put_space@unpacker@@QEAAPEAC_K@Z 000000014000c678 f   unpack.obj
 0001:0000b6c4       ?put_stackmap_type@unpacker@@QEAAXXZ 000000014000c6c4 f   unpack.obj
 0001:0000b760       ?putlayout@unpacker@@QEAAXPEAPEAUband@@@Z 000000014000c760 f   unpack.obj
 0001:0000b99c       ?putref@unpacker@@QEAAXPEAUentry@@@Z 000000014000c99c f   unpack.obj
 0001:0000b9f4       ?putref_index@unpacker@@QEAAHPEAUentry@@H@Z 000000014000c9f4 f   unpack.obj
 0001:0000baa4       ?putu1ref@unpacker@@QEAAXPEAUentry@@@Z 000000014000caa4 f   unpack.obj
 0001:0000bad8       ?putu2@unpacker@@QEAAXH@Z  000000014000cad8 f   unpack.obj
 0001:0000bb18       ?putu4@unpacker@@QEAAXH@Z  000000014000cb18 f   unpack.obj
 0001:0000bb4c       ?putu8@unpacker@@QEAAX_J@Z 000000014000cb4c f   unpack.obj
 0001:0000bbac       ?readBandData@attr_definitions@unpacker@@QEAAXH@Z 000000014000cbac f   unpack.obj
 0001:0000bca0       ?readBandData@attr_definitions@unpacker@@QEAAXPEAPEAUband@@I@Z 000000014000cca0 f   unpack.obj
 0001:0000be14       ?read_Utf8_values@unpacker@@QEAAXPEAUentry@@HC@Z 000000014000ce14 f i unpack.obj
 0001:0000c568       ?read_attr_defs@unpacker@@QEAAXXZ 000000014000d568 f   unpack.obj
 0001:0000c8b4       ?read_attrs@unpacker@@QEAAXHH@Z 000000014000d8b4 f   unpack.obj
 0001:0000d59c       ?read_bands@unpacker@@QEAAXXZ 000000014000e59c f   unpack.obj
 0001:0000d624       ?read_bcs@unpacker@@QEAAXXZ 000000014000e624 f i unpack.obj
 0001:0000d9f0       ?read_bootstrap_methods@unpacker@@QEAAXPEAUentry@@HC@Z 000000014000e9f0 f   unpack.obj
 0001:0000db80       ?read_classes@unpacker@@QEAAXXZ 000000014000eb80 f   unpack.obj
 0001:0000dcf8       ?read_code_headers@unpacker@@QEAAXXZ 000000014000ecf8 f   unpack.obj
 0001:0000de94       ?read_cp@unpacker@@QEAAXXZ 000000014000ee94 f   unpack.obj
 0001:0000e208       ?read_double_refs@unpacker@@QEAAXAEAUband@@CCPEAUentry@@HC@Z 000000014000f208 f   unpack.obj
 0001:0000e31c       ?read_double_words@unpacker@@QEAAXAEAUband@@PEAUentry@@HCH@Z 000000014000f31c f   unpack.obj
 0001:0000e3d4       ?read_file_header@unpacker@@QEAAXXZ 000000014000f3d4 f   unpack.obj
 0001:0000ed8c       ?read_files@unpacker@@QEAAXXZ 000000014000fd8c f   unpack.obj
 0001:0000eeac       ?read_ics@unpacker@@QEAAXXZ 000000014000feac f   unpack.obj
 0001:0000f304       ?read_method_handle@unpacker@@QEAAXPEAUentry@@HCH@Z 0000000140010304 f   unpack.obj
 0001:0000f440       ?read_method_type@unpacker@@QEAAXPEAUentry@@HCH@Z 0000000140010440 f   unpack.obj
 0001:0000f558       ?read_signature_values@unpacker@@QEAAXPEAUentry@@HC@Z 0000000140010558 f   unpack.obj
 0001:0000f724       ?read_single_refs@unpacker@@QEAAXAEAUband@@CPEAUentry@@HCH@Z 0000000140010724 f   unpack.obj
 0001:0000f858       ?read_single_words@unpacker@@QEAAXAEAUband@@PEAUentry@@HCH@Z 0000000140010858 f i unpack.obj
 0001:0000f904       ?redirect_stdio@unpacker@@QEAAXXZ 0000000140010904 f   unpack.obj
 0001:0000f9f4       ?ref_band_for_op@unpacker@@QEAAPEAUband@@H@Z 00000001400109f4 f   unpack.obj
 0001:0000fb54       ?ref_band_for_self_op@unpacker@@QEAAPEAUband@@HAEA_NAEAH@Z 0000000140010b54 f   unpack.obj
 0001:0000fbb4       ?requestOutputIndex@entry@@QEAAXAEAUcpool@@H@Z 0000000140010bb4 f   unpack.obj
 0001:0000fc58       ?reset@unpacker@@QEAAXXZ   0000000140010c58 f   unpack.obj
 0001:0000fefc       ?resetOutputIndexes@cpool@@QEAAXXZ 0000000140010efc f   unpack.obj
 0001:0000ff68       ?reset_cur_classfile@unpacker@@QEAAXXZ 0000000140010f68 f   unpack.obj
 0001:0000ffc0       ?saveTo@unpacker@@QEAAXAEAUbytes@@PEAC_K@Z 0000000140010fc0 f   unpack.obj
 0001:00010050       ?set_option@unpacker@@QEAA_NPEBD0@Z 0000000140011050 f   unpack.obj
 0001:00010200       ?start@unpacker@@QEAAXPEAX_K@Z 0000000140011200 f   unpack.obj
 0001:00010294       ?to_bci@unpacker@@QEAAII@Z 0000000140011294 f   unpack.obj
 0001:00010304       ?typeSize@entry@@QEAAHXZ   0000000140011304 f   unpack.obj
 0001:000103a8       ?write_attrs@unpacker@@QEAAHH_K@Z 00000001400113a8 f   unpack.obj
 0001:0001100c       ?write_bc_ops@unpacker@@QEAAXXZ 000000014001200c f i unpack.obj
 0001:000119f0       ?write_bsms@unpacker@@QEAAHHH@Z 00000001400129f0 f   unpack.obj
 0001:00011b84       ?write_classfile_head@unpacker@@QEAAXXZ 0000000140012b84 f   unpack.obj
 0001:00011d68       ?write_classfile_tail@unpacker@@QEAAXXZ 0000000140012d68 f   unpack.obj
 0001:00012050       ?write_code@unpacker@@QEAAXXZ 0000000140013050 f i unpack.obj
 0001:0001226c       ?write_file_to_jar@unpacker@@QEAAXPEAUfile@1@@Z 000000014001326c f   unpack.obj
 0001:0001244c       ?write_ics@unpacker@@QEAAHHH@Z 000000014001344c f   unpack.obj
 0001:00012824       ?write_members@unpacker@@QEAAXHH@Z 0000000140013824 f   unpack.obj
 0001:0001299c       _snprintf                  000000014001399c f i unpack.obj
 0001:000129f4       outputEntry_cmp            00000001400139f4 f   unpack.obj
 0001:00012a60       raw_address_cmp            0000000140013a60 f   unpack.obj
 0001:00012a74       ?must_calloc@@YAPEAX_K0@Z  0000000140013a74 f   utils.obj
 0001:00012ad4       ?unpack_abort@@YAXPEBDPEAUunpacker@@@Z 0000000140013ad4 f   utils.obj
 0001:00012b2c       ?unpack_aborting@@YA_NPEAUunpacker@@@Z 0000000140013b2c f   utils.obj
 0001:00012b70       ?addJarEntry@jar@@QEAAXPEBD_NHAEAUbytes@@2@Z 0000000140013b70 f   zip.obj
 0001:00012cc8       ?add_to_jar_directory@jar@@QEAAXPEBD_NHHHK@Z 0000000140013cc8 f   zip.obj
 0001:00012e4c       ?closeJarFile@jar@@QEAAX_N@Z 0000000140013e4c f   zip.obj
 0001:00012ecc       ?deflate_bytes@jar@@QEAA_NAEAUbytes@@0@Z 0000000140013ecc f   zip.obj
 0001:0001301c       ?dostime@jar@@QEAAKHHHHHH@Z 000000014001401c f i zip.obj
 0001:00013080       ?free@gunzip@@QEAAXXZ      0000000140014080 f   zip.obj
 0001:000130c8       ?get_dostime@jar@@QEAAKH@Z 00000001400140c8 f   zip.obj
 0001:000131d0       ?init@gunzip@@QEAAXPEAUunpacker@@@Z 00000001400141d0 f   zip.obj
 0001:00013258       ?init@jar@@QEAAXPEAUunpacker@@@Z 0000000140014258 f   zip.obj
 0001:00013288       ?openJarFile@jar@@QEAAXPEBD@Z 0000000140014288 f   zip.obj
 0001:000132ec       ?read_fixed_field@gunzip@@QEAAXPEAD_K@Z 00000001400142ec f   zip.obj
 0001:0001359c       ?start@gunzip@@QEAAXH@Z    000000014001459c f   zip.obj
 0001:000136b0       ?write_central_directory@jar@@QEAAXXZ 00000001400146b0 f   zip.obj
 0001:0001383c       ?write_data@jar@@QEAAXPEAX_K@Z 000000014001483c f   zip.obj
 0001:000138bc       ?write_jar_extra@jar@@QEAAXHHI@Z 00000001400148bc f   zip.obj
 0001:00013924       ?write_jar_header@jar@@QEAAXPEBD_NHHHI@Z 0000000140014924 f   zip.obj
 0001:00013a8c       __raise_securityfailure    0000000140014a8c f   MSVCRT:gs_report.obj
 0001:00013ac0       __report_gsfailure         0000000140014ac0 f   MSVCRT:gs_report.obj
 0001:00013b94       __report_rangecheckfailure 0000000140014b94 f   MSVCRT:gs_report.obj
 0001:00013ba8       __report_securityfailure   0000000140014ba8 f   MSVCRT:gs_report.obj
 0001:00013d28       __GSHandlerCheck           0000000140014d28 f   MSVCRT:gshandler.obj
 0001:00013d48       __GSHandlerCheckCommon     0000000140014d48 f   MSVCRT:gshandler.obj
 0001:00013dc0       __security_check_cookie    0000000140014dc0 f   MSVCRT:amdsecgs.obj
 0001:00013df0       __chkstk                   0000000140014df0 f   MSVCRT:chkstk.obj
 0001:00013df0       _alloca_probe              0000000140014df0 f   MSVCRT:chkstk.obj
 0001:000140a0       mainCRTStartup             00000001400150a0 f   MSVCRT:exe_main.obj
 0001:000140b4       __scrt_acquire_startup_lock 00000001400150b4 f   MSVCRT:utility.obj
 0001:000140f0       __scrt_initialize_crt      00000001400150f0 f   MSVCRT:utility.obj
 0001:0001413c       __scrt_initialize_onexit_tables 000000014001513c f   MSVCRT:utility.obj
 0001:000141c8       __scrt_is_nonwritable_in_current_image 00000001400151c8 f   MSVCRT:utility.obj
 0001:00014260       __scrt_release_startup_lock 0000000140015260 f   MSVCRT:utility.obj
 0001:00014284       __scrt_uninitialize_crt    0000000140015284 f   MSVCRT:utility.obj
 0001:000142b0       _onexit                    00000001400152b0 f   MSVCRT:utility.obj
 0001:000142ec       atexit                     00000001400152ec f   MSVCRT:utility.obj
 0001:00014304       __security_init_cookie     0000000140015304 f   MSVCRT:gs_support.obj
 0001:000143b0       __scrt_exe_initialize_mta  00000001400153b0 f   MSVCRT:utility_desktop.obj
 0001:000143b0       __scrt_initialize_winrt    00000001400153b0 f   MSVCRT:utility_desktop.obj
 0001:000143b0       __scrt_stub_for_initialize_mta 00000001400153b0 f   MSVCRT:utility_desktop.obj
 0001:000143b0       _get_startup_commit_mode   00000001400153b0 f   MSVCRT:commit_mode.obj
 0001:000143b0       _get_startup_new_mode      00000001400153b0 f   MSVCRT:new_mode.obj
 0001:000143b0       _get_startup_thread_locale_mode 00000001400153b0 f   MSVCRT:thread_locale.obj
 0001:000143b0       _matherr                   00000001400153b0 f   MSVCRT:matherr.obj
 0001:000143b4       _get_startup_argv_mode     00000001400153b4 f   MSVCRT:argv_mode.obj
 0001:000143bc       _get_startup_file_mode     00000001400153bc f   MSVCRT:file_mode.obj
 0001:000143c4       ?__scrt_initialize_type_info@@YAXXZ 00000001400153c4 f   MSVCRT:tncleanup.obj
 0001:000143d4       __acrt_initialize          00000001400153d4 f   MSVCRT:ucrt_stubs.obj
 0001:000143d4       __acrt_uninitialize        00000001400153d4 f   MSVCRT:ucrt_stubs.obj
 0001:000143d4       __scrt_stub_for_acrt_initialize 00000001400153d4 f   MSVCRT:ucrt_stubs.obj
 0001:000143d4       __scrt_stub_for_acrt_uninitialize 00000001400153d4 f   MSVCRT:ucrt_stubs.obj
 0001:000143d4       __vcrt_initialize          00000001400153d4 f   MSVCRT:ucrt_stubs.obj
 0001:000143d4       __vcrt_uninitialize        00000001400153d4 f   MSVCRT:ucrt_stubs.obj
 0001:000143d4       _should_initialize_environment 00000001400153d4 f   MSVCRT:env_mode.obj
 0001:000143d8       _guard_check_icall_nop     00000001400153d8 f   MSVCRT:guard_support.obj
 0001:000143d8       _initialize_denormal_control 00000001400153d8 f   MSVCRT:denormal_control.obj
 0001:000143d8       _initialize_invalid_parameter_handler 00000001400153d8 f   MSVCRT:invalid_parameter_handler.obj
 0001:000143dc       __local_stdio_scanf_options 00000001400153dc f i MSVCRT:default_local_stdio_options.obj
 0001:000143e4       __scrt_initialize_default_local_stdio_options 00000001400153e4 f   MSVCRT:default_local_stdio_options.obj
 0001:00014400       __scrt_is_user_matherr_present 0000000140015400 f   MSVCRT:matherr_detection.obj
 0001:0001440c       __scrt_get_dyn_tls_init_callback 000000014001540c f   MSVCRT:dyn_tls_init.obj
 0001:00014414       __scrt_get_dyn_tls_dtor_callback 0000000140015414 f   MSVCRT:dyn_tls_dtor.obj
 0001:0001441c       __crt_debugger_hook        000000014001541c f   MSVCRT:utility_desktop.obj
 0001:00014424       __scrt_fastfail            0000000140015424 f   MSVCRT:utility_desktop.obj
 0001:00014570       __scrt_initialize_mta      0000000140015570 f   MSVCRT:utility_desktop.obj
 0001:00014578       __scrt_is_managed_app      0000000140015578 f   MSVCRT:utility_desktop.obj
 0001:000145cc       __scrt_set_unhandled_exception_filter 00000001400155cc f   MSVCRT:utility_desktop.obj
 0001:000145dc       __scrt_unhandled_exception_filter 00000001400155dc f   MSVCRT:utility_desktop.obj
 0001:00014638       _RTC_Initialize            0000000140015638 f   MSVCRT:initsect.obj
 0001:00014674       _RTC_Terminate             0000000140015674 f   MSVCRT:initsect.obj
 0001:000146b0       __isa_available_init       00000001400156b0 f   MSVCRT:cpu_disp.obj
 0001:0001485c       __scrt_is_ucrt_dll_in_use  000000014001585c f   MSVCRT:ucrt_detection.obj
 0001:00014870       memcpy                     0000000140015870 f   vcruntime:VCRUNTIME140.dll
 0001:00014876       memset                     0000000140015876 f   vcruntime:VCRUNTIME140.dll
 0001:0001487c       memcmp                     000000014001587c f   vcruntime:VCRUNTIME140.dll
 0001:00014882       strchr                     0000000140015882 f   vcruntime:VCRUNTIME140.dll
 0001:00014888       strrchr                    0000000140015888 f   vcruntime:VCRUNTIME140.dll
 0001:0001488e       __C_specific_handler       000000014001588e f   vcruntime:VCRUNTIME140.dll
 0001:00014894       __current_exception        0000000140015894 f   vcruntime:VCRUNTIME140.dll
 0001:0001489a       __current_exception_context 000000014001589a f   vcruntime:VCRUNTIME140.dll
 0001:000148a0       strcmp                     00000001400158a0 f   ucrt:api-ms-win-crt-string-l1-1-0.dll
 0001:000148a6       strlen                     00000001400158a6 f   ucrt:api-ms-win-crt-string-l1-1-0.dll
 0001:000148ac       exit                       00000001400158ac f   ucrt:api-ms-win-crt-runtime-l1-1-0.dll
 0001:000148b2       strcat                     00000001400158b2 f   ucrt:api-ms-win-crt-string-l1-1-0.dll
 0001:000148b8       _seh_filter_exe            00000001400158b8 f   ucrt:api-ms-win-crt-runtime-l1-1-0.dll
 0001:000148be       _set_app_type              00000001400158be f   ucrt:api-ms-win-crt-runtime-l1-1-0.dll
 0001:000148c4       __setusermatherr           00000001400158c4 f   ucrt:api-ms-win-crt-math-l1-1-0.dll
 0001:000148ca       _configure_narrow_argv     00000001400158ca f   ucrt:api-ms-win-crt-runtime-l1-1-0.dll
 0001:000148d0       _initialize_narrow_environment 00000001400158d0 f   ucrt:api-ms-win-crt-runtime-l1-1-0.dll
 0001:000148d6       _get_initial_narrow_environment 00000001400158d6 f   ucrt:api-ms-win-crt-runtime-l1-1-0.dll
 0001:000148dc       _initterm                  00000001400158dc f   ucrt:api-ms-win-crt-runtime-l1-1-0.dll
 0001:000148e2       _initterm_e                00000001400158e2 f   ucrt:api-ms-win-crt-runtime-l1-1-0.dll
 0001:000148e8       _exit                      00000001400158e8 f   ucrt:api-ms-win-crt-runtime-l1-1-0.dll
 0001:000148ee       _set_fmode                 00000001400158ee f   ucrt:api-ms-win-crt-stdio-l1-1-0.dll
 0001:000148f4       __p___argc                 00000001400158f4 f   ucrt:api-ms-win-crt-runtime-l1-1-0.dll
 0001:000148fa       __p___argv                 00000001400158fa f   ucrt:api-ms-win-crt-runtime-l1-1-0.dll
 0001:00014900       _cexit                     0000000140015900 f   ucrt:api-ms-win-crt-runtime-l1-1-0.dll
 0001:00014906       _c_exit                    0000000140015906 f   ucrt:api-ms-win-crt-runtime-l1-1-0.dll
 0001:0001490c       _register_thread_local_exe_atexit_callback 000000014001590c f   ucrt:api-ms-win-crt-runtime-l1-1-0.dll
 0001:00014912       _configthreadlocale        0000000140015912 f   ucrt:api-ms-win-crt-locale-l1-1-0.dll
 0001:00014918       _set_new_mode              0000000140015918 f   ucrt:api-ms-win-crt-heap-l1-1-0.dll
 0001:0001491e       __p__commode               000000014001591e f   ucrt:api-ms-win-crt-stdio-l1-1-0.dll
 0001:00014924       _initialize_onexit_table   0000000140015924 f   ucrt:api-ms-win-crt-runtime-l1-1-0.dll
 0001:0001492a       _register_onexit_function  000000014001592a f   ucrt:api-ms-win-crt-runtime-l1-1-0.dll
 0001:00014930       _crt_atexit                0000000140015930 f   ucrt:api-ms-win-crt-runtime-l1-1-0.dll
 0001:00014936       terminate                  0000000140015936 f   ucrt:api-ms-win-crt-runtime-l1-1-0.dll
 0001:00014950       _guard_dispatch_icall_nop  0000000140015950 f   MSVCRT:guard_dispatch.obj
 0001:00014970       _guard_xfg_dispatch_icall_nop 0000000140015970 f   MSVCRT:guard_xfg_dispatch.obj
 0002:00000000       __imp_RtlCaptureContext    0000000140016000     kernel32:KERNEL32.dll
 0002:00000008       __imp_RtlLookupFunctionEntry 0000000140016008     kernel32:KERNEL32.dll
 0002:00000010       __imp_RtlVirtualUnwind     0000000140016010     kernel32:KERNEL32.dll
 0002:00000018       __imp_UnhandledExceptionFilter 0000000140016018     kernel32:KERNEL32.dll
 0002:00000020       __imp_SetUnhandledExceptionFilter 0000000140016020     kernel32:KERNEL32.dll
 0002:00000028       __imp_GetCurrentProcess    0000000140016028     kernel32:KERNEL32.dll
 0002:00000030       __imp_TerminateProcess     0000000140016030     kernel32:KERNEL32.dll
 0002:00000038       __imp_IsProcessorFeaturePresent 0000000140016038     kernel32:KERNEL32.dll
 0002:00000040       __imp_QueryPerformanceCounter 0000000140016040     kernel32:KERNEL32.dll
 0002:00000048       __imp_GetCurrentProcessId  0000000140016048     kernel32:KERNEL32.dll
 0002:00000050       __imp_GetCurrentThreadId   0000000140016050     kernel32:KERNEL32.dll
 0002:00000058       __imp_GetSystemTimeAsFileTime 0000000140016058     kernel32:KERNEL32.dll
 0002:00000060       __imp_InitializeSListHead  0000000140016060     kernel32:KERNEL32.dll
 0002:00000068       __imp_IsDebuggerPresent    0000000140016068     kernel32:KERNEL32.dll
 0002:00000070       __imp_GetModuleHandleW     0000000140016070     kernel32:KERNEL32.dll
 0002:00000078       \177KERNEL32_NULL_THUNK_DATA 0000000140016078     kernel32:KERNEL32.dll
 0002:00000080       __imp_memcpy               0000000140016080     vcruntime:VCRUNTIME140.dll
 0002:00000088       __imp_memset               0000000140016088     vcruntime:VCRUNTIME140.dll
 0002:00000090       __imp_memcmp               0000000140016090     vcruntime:VCRUNTIME140.dll
 0002:00000098       __imp_strchr               0000000140016098     vcruntime:VCRUNTIME140.dll
 0002:000000a0       __imp_strrchr              00000001400160a0     vcruntime:VCRUNTIME140.dll
 0002:000000a8       __imp___C_specific_handler 00000001400160a8     vcruntime:VCRUNTIME140.dll
 0002:000000b0       __imp___current_exception  00000001400160b0     vcruntime:VCRUNTIME140.dll
 0002:000000b8       __imp___current_exception_context 00000001400160b8     vcruntime:VCRUNTIME140.dll
 0002:000000c0       \177VCRUNTIME140_NULL_THUNK_DATA 00000001400160c0     vcruntime:VCRUNTIME140.dll
 0002:000000c8       __imp_atoi                 00000001400160c8     ucrt:api-ms-win-crt-convert-l1-1-0.dll
 0002:000000d0       \177api-ms-win-crt-convert-l1-1-0_NULL_THUNK_DATA 00000001400160d0     ucrt:api-ms-win-crt-convert-l1-1-0.dll
 0002:000000d8       __imp_getenv               00000001400160d8     ucrt:api-ms-win-crt-environment-l1-1-0.dll
 0002:000000e0       \177api-ms-win-crt-environment-l1-1-0_NULL_THUNK_DATA 00000001400160e0     ucrt:api-ms-win-crt-environment-l1-1-0.dll
 0002:000000e8       __imp_remove               00000001400160e8     ucrt:api-ms-win-crt-filesystem-l1-1-0.dll
 0002:000000f0       \177api-ms-win-crt-filesystem-l1-1-0_NULL_THUNK_DATA 00000001400160f0     ucrt:api-ms-win-crt-filesystem-l1-1-0.dll
 0002:000000f8       __imp_malloc               00000001400160f8     ucrt:api-ms-win-crt-heap-l1-1-0.dll
 0002:00000100       __imp_free                 0000000140016100     ucrt:api-ms-win-crt-heap-l1-1-0.dll
 0002:00000108       __imp__set_new_mode        0000000140016108     ucrt:api-ms-win-crt-heap-l1-1-0.dll
 0002:00000110       __imp_calloc               0000000140016110     ucrt:api-ms-win-crt-heap-l1-1-0.dll
 0002:00000118       __imp_realloc              0000000140016118     ucrt:api-ms-win-crt-heap-l1-1-0.dll
 0002:00000120       \177api-ms-win-crt-heap-l1-1-0_NULL_THUNK_DATA 0000000140016120     ucrt:api-ms-win-crt-heap-l1-1-0.dll
 0002:00000128       __imp__configthreadlocale  0000000140016128     ucrt:api-ms-win-crt-locale-l1-1-0.dll
 0002:00000130       \177api-ms-win-crt-locale-l1-1-0_NULL_THUNK_DATA 0000000140016130     ucrt:api-ms-win-crt-locale-l1-1-0.dll
 0002:00000138       __imp___setusermatherr     0000000140016138     ucrt:api-ms-win-crt-math-l1-1-0.dll
 0002:00000140       \177api-ms-win-crt-math-l1-1-0_NULL_THUNK_DATA 0000000140016140     ucrt:api-ms-win-crt-math-l1-1-0.dll
 0002:00000148       __imp_terminate            0000000140016148     ucrt:api-ms-win-crt-runtime-l1-1-0.dll
 0002:00000150       __imp__crt_atexit          0000000140016150     ucrt:api-ms-win-crt-runtime-l1-1-0.dll
 0002:00000158       __imp__register_onexit_function 0000000140016158     ucrt:api-ms-win-crt-runtime-l1-1-0.dll
 0002:00000160       __imp__initialize_onexit_table 0000000140016160     ucrt:api-ms-win-crt-runtime-l1-1-0.dll
 0002:00000168       __imp_abort                0000000140016168     ucrt:api-ms-win-crt-runtime-l1-1-0.dll
 0002:00000170       __imp__errno               0000000140016170     ucrt:api-ms-win-crt-runtime-l1-1-0.dll
 0002:00000178       __imp__register_thread_local_exe_atexit_callback 0000000140016178     ucrt:api-ms-win-crt-runtime-l1-1-0.dll
 0002:00000180       __imp__c_exit              0000000140016180     ucrt:api-ms-win-crt-runtime-l1-1-0.dll
 0002:00000188       __imp__cexit               0000000140016188     ucrt:api-ms-win-crt-runtime-l1-1-0.dll
 0002:00000190       __imp__seh_filter_exe      0000000140016190     ucrt:api-ms-win-crt-runtime-l1-1-0.dll
 0002:00000198       __imp__set_app_type        0000000140016198     ucrt:api-ms-win-crt-runtime-l1-1-0.dll
 0002:000001a0       __imp_exit                 00000001400161a0     ucrt:api-ms-win-crt-runtime-l1-1-0.dll
 0002:000001a8       __imp__configure_narrow_argv 00000001400161a8     ucrt:api-ms-win-crt-runtime-l1-1-0.dll
 0002:000001b0       __imp__initialize_narrow_environment 00000001400161b0     ucrt:api-ms-win-crt-runtime-l1-1-0.dll
 0002:000001b8       __imp__get_initial_narrow_environment 00000001400161b8     ucrt:api-ms-win-crt-runtime-l1-1-0.dll
 0002:000001c0       __imp__initterm            00000001400161c0     ucrt:api-ms-win-crt-runtime-l1-1-0.dll
 0002:000001c8       __imp__initterm_e          00000001400161c8     ucrt:api-ms-win-crt-runtime-l1-1-0.dll
 0002:000001d0       __imp__exit                00000001400161d0     ucrt:api-ms-win-crt-runtime-l1-1-0.dll
 0002:000001d8       __imp___p___argv           00000001400161d8     ucrt:api-ms-win-crt-runtime-l1-1-0.dll
 0002:000001e0       __imp___p___argc           00000001400161e0     ucrt:api-ms-win-crt-runtime-l1-1-0.dll
 0002:000001e8       \177api-ms-win-crt-runtime-l1-1-0_NULL_THUNK_DATA 00000001400161e8     ucrt:api-ms-win-crt-runtime-l1-1-0.dll
 0002:000001f0       __imp_fwrite               00000001400161f0     ucrt:api-ms-win-crt-stdio-l1-1-0.dll
 0002:000001f8       __imp_fseek                00000001400161f8     ucrt:api-ms-win-crt-stdio-l1-1-0.dll
 0002:00000200       __imp_fclose               0000000140016200     ucrt:api-ms-win-crt-stdio-l1-1-0.dll
 0002:00000208       __imp___stdio_common_vsprintf 0000000140016208     ucrt:api-ms-win-crt-stdio-l1-1-0.dll
 0002:00000210       __imp___p__commode         0000000140016210     ucrt:api-ms-win-crt-stdio-l1-1-0.dll
 0002:00000218       __imp___acrt_iob_func      0000000140016218     ucrt:api-ms-win-crt-stdio-l1-1-0.dll
 0002:00000220       __imp__set_fmode           0000000140016220     ucrt:api-ms-win-crt-stdio-l1-1-0.dll
 0002:00000228       __imp_fopen                0000000140016228     ucrt:api-ms-win-crt-stdio-l1-1-0.dll
 0002:00000230       __imp_fread                0000000140016230     ucrt:api-ms-win-crt-stdio-l1-1-0.dll
 0002:00000238       __imp___stdio_common_vfprintf 0000000140016238     ucrt:api-ms-win-crt-stdio-l1-1-0.dll
 0002:00000240       __imp__fileno              0000000140016240     ucrt:api-ms-win-crt-stdio-l1-1-0.dll
 0002:00000240       __imp_fileno               0000000140016240     ucrt:api-ms-win-crt-stdio-l1-1-0.dll
 0002:00000248       __imp_fflush               0000000140016248     ucrt:api-ms-win-crt-stdio-l1-1-0.dll
 0002:00000250       \177api-ms-win-crt-stdio-l1-1-0_NULL_THUNK_DATA 0000000140016250     ucrt:api-ms-win-crt-stdio-l1-1-0.dll
 0002:00000258       __imp__strdup              0000000140016258     ucrt:api-ms-win-crt-string-l1-1-0.dll
 0002:00000258       __imp_strdup               0000000140016258     ucrt:api-ms-win-crt-string-l1-1-0.dll
 0002:00000260       __imp_strncmp              0000000140016260     ucrt:api-ms-win-crt-string-l1-1-0.dll
 0002:00000268       __imp_strlen               0000000140016268     ucrt:api-ms-win-crt-string-l1-1-0.dll
 0002:00000270       __imp_strncat              0000000140016270     ucrt:api-ms-win-crt-string-l1-1-0.dll
 0002:00000278       __imp_strcat               0000000140016278     ucrt:api-ms-win-crt-string-l1-1-0.dll
 0002:00000280       __imp_strtok               0000000140016280     ucrt:api-ms-win-crt-string-l1-1-0.dll
 0002:00000288       __imp_strcmp               0000000140016288     ucrt:api-ms-win-crt-string-l1-1-0.dll
 0002:00000290       \177api-ms-win-crt-string-l1-1-0_NULL_THUNK_DATA 0000000140016290     ucrt:api-ms-win-crt-string-l1-1-0.dll
 0002:00000298       __imp__gmtime64            0000000140016298     ucrt:api-ms-win-crt-time-l1-1-0.dll
 0002:000002a0       __imp__time64              00000001400162a0     ucrt:api-ms-win-crt-time-l1-1-0.dll
 0002:000002a8       \177api-ms-win-crt-time-l1-1-0_NULL_THUNK_DATA 00000001400162a8     ucrt:api-ms-win-crt-time-l1-1-0.dll
 0002:000002b0       __imp_qsort                00000001400162b0     ucrt:api-ms-win-crt-utility-l1-1-0.dll
 0002:000002b8       \177api-ms-win-crt-utility-l1-1-0_NULL_THUNK_DATA 00000001400162b8     ucrt:api-ms-win-crt-utility-l1-1-0.dll
 0002:000002c0       __guard_check_icall_fptr   00000001400162c0     MSVCRT:guard_support.obj
 0002:000002c8       __guard_xfg_check_icall_fptr 00000001400162c8     MSVCRT:guard_support.obj
 0002:000002d0       __guard_dispatch_icall_fptr 00000001400162d0     MSVCRT:guard_support.obj
 0002:000002d8       __guard_xfg_dispatch_icall_fptr 00000001400162d8     MSVCRT:guard_support.obj
 0002:000002e0       __guard_xfg_table_dispatch_icall_fptr 00000001400162e0     MSVCRT:guard_support.obj
 0002:000002e8       __castguard_check_failure_os_handled_fptr 00000001400162e8     MSVCRT:guard_support.obj
 0002:000002f0       __guard_memcpy_fptr        00000001400162f0     vcruntime:softmemtag.obj
 0002:000002f8       __xc_a                     00000001400162f8     MSVCRT:initializers.obj
 0002:00000308       __xc_z                     0000000140016308     MSVCRT:initializers.obj
 0002:00000310       __xi_a                     0000000140016310     MSVCRT:initializers.obj
 0002:00000328       __xi_z                     0000000140016328     MSVCRT:initializers.obj
 0002:00000330       __xp_a                     0000000140016330     MSVCRT:initializers.obj
 0002:00000338       __xp_z                     0000000140016338     MSVCRT:initializers.obj
 0002:00000340       __xt_a                     0000000140016340     MSVCRT:initializers.obj
 0002:00000348       __xt_z                     0000000140016348     MSVCRT:initializers.obj
 0002:00000350       ??_C@_05OJPKCACG@1?43?41@  0000000140016350     compress.obj
 0002:00000360       deflate_copyright          0000000140016360     deflate.obj
 0002:00000cf8       ??_C@_0BD@PJCBIDD@invalid?5block?5type@ 0000000140016cf8     infback.obj
 0002:00000d10       ??_C@_0BN@LGAADGOK@invalid?5stored?5block?5lengths@ 0000000140016d10     infback.obj
 0002:00000d30       ??_C@_0CE@GMIGFPBB@too?5many?5length?5or?5distance?5sym@ 0000000140016d30     infback.obj
 0002:00000d58       ??_C@_0BJ@HDEPPGOH@invalid?5code?5lengths?5set@ 0000000140016d58     infback.obj
 0002:00000d78       ??_C@_0BK@BMMPFBBH@invalid?5bit?5length?5repeat@ 0000000140016d78     infback.obj
 0002:00000d98       ??_C@_0CF@DGDMADCD@invalid?5code?5?9?9?5missing?5end?9of?9@ 0000000140016d98     infback.obj
 0002:00000dc0       ??_C@_0BM@IIMGAINC@invalid?5literal?1lengths?5set@ 0000000140016dc0     infback.obj
 0002:00000de0       ??_C@_0BG@GMDFCBGP@invalid?5distances?5set@ 0000000140016de0     infback.obj
 0002:00000df8       ??_C@_0BM@FFFLPBBC@invalid?5literal?1length?5code@ 0000000140016df8     infback.obj
 0002:00000e18       ??_C@_0BG@LBKINIKP@invalid?5distance?5code@ 0000000140016e18     infback.obj
 0002:00000e30       ??_C@_0BO@ECPMAOGG@invalid?5distance?5too?5far?5back@ 0000000140016e30     infback.obj
 0002:000016f8       ??_C@_0BH@LIBMMIGA@incorrect?5header?5check@ 00000001400176f8     inflate.obj
 0002:00001710       ??_C@_0BL@IHKGDAEE@unknown?5compression?5method@ 0000000140017710     inflate.obj
 0002:00001730       ??_C@_0BE@EMOGCLGO@invalid?5window?5size@ 0000000140017730     inflate.obj
 0002:00001748       ??_C@_0BJ@BLBBCOMO@unknown?5header?5flags?5set@ 0000000140017748     inflate.obj
 0002:00001768       ??_C@_0BE@GONKLEPM@header?5crc?5mismatch@ 0000000140017768     inflate.obj
 0002:00001780       ??_C@_0BF@MEIGEHBE@incorrect?5data?5check@ 0000000140017780     inflate.obj
 0002:00001798       ??_C@_0BH@FGKKJGOC@incorrect?5length?5check@ 0000000140017798     inflate.obj
 0002:000017b0       inflate_copyright          00000001400177b0     inftrees.obj
 0002:000018e0       _length_code               00000001400178e0     trees.obj
 0002:000019e0       _dist_code                 00000001400179e0     trees.obj
 0002:00004c30       z_errmsg                   000000014001ac30     zutil.obj
 0002:00004c80       ??_C@_0BA@MOKMMFOD@need?5dictionary@ 000000014001ac80     zutil.obj
 0002:00004c90       ??_C@_0L@FNAOCBOG@stream?5end@ 000000014001ac90     zutil.obj
 0002:00004c9b       ??_C@_00CNPNBAHC@@         000000014001ac9b     zutil.obj
 0002:00004ca0       ??_C@_0L@KIJFAKBJ@file?5error@ 000000014001aca0     zutil.obj
 0002:00004cb0       ??_C@_0N@MKKNPMJD@stream?5error@ 000000014001acb0     zutil.obj
 0002:00004cc0       ??_C@_0L@HAHMBNLP@data?5error@ 000000014001acc0     zutil.obj
 0002:00004cd0       ??_C@_0BE@OGGJBMCE@insufficient?5memory@ 000000014001acd0     zutil.obj
 0002:00004ce8       ??_C@_0N@DFPGLBGC@buffer?5error@ 000000014001ace8     zutil.obj
 0002:00004cf8       ??_C@_0BF@CJFPCCEG@incompatible?5version@ 000000014001acf8     zutil.obj
 0002:00005bb0       ??_C@_0P@NFDCFGCL@cp_Utf8_prefix@ 000000014001bbb0     bands.obj
 0002:00005bc0       ??_C@_0P@LOHPAGNO@cp_Utf8_suffix@ 000000014001bbc0     bands.obj
 0002:00005bd0       ??_C@_0O@IHLLKPBK@cp_Utf8_chars@ 000000014001bbd0     bands.obj
 0002:00005be0       ??_C@_0BD@EOIEJGOP@cp_Utf8_big_suffix@ 000000014001bbe0     bands.obj
 0002:00005bf8       ??_C@_0BC@HDLINKIK@cp_Utf8_big_chars@ 000000014001bbf8     bands.obj
 0002:00005c0c       ??_C@_06IGKKGOEN@cp_Int@   000000014001bc0c     bands.obj
 0002:00005c18       ??_C@_08OBBFNHHD@cp_Float@ 000000014001bc18     bands.obj
 0002:00005c28       ??_C@_0L@HNFJMOEO@cp_Long_hi@ 000000014001bc28     bands.obj
 0002:00005c38       ??_C@_0L@CMAKMBBE@cp_Long_lo@ 000000014001bc38     bands.obj
 0002:00005c48       ??_C@_0N@CPNNOOPC@cp_Double_hi@ 000000014001bc48     bands.obj
 0002:00005c58       ??_C@_0N@HOIOOBKI@cp_Double_lo@ 000000014001bc58     bands.obj
 0002:00005c68       ??_C@_09HFEHKGNE@cp_String@ 000000014001bc68     bands.obj
 0002:00005c78       ??_C@_08BOENACK@cp_Class@  000000014001bc78     bands.obj
 0002:00005c88       ??_C@_0BC@FENMLAPO@cp_Signature_form@ 000000014001bc88     bands.obj
 0002:00005ca0       ??_C@_0BF@MEOEAPGK@cp_Signature_classes@ 000000014001bca0     bands.obj
 0002:00005cb8       ??_C@_0O@JHMEINNJ@cp_Descr_name@ 000000014001bcb8     bands.obj
 0002:00005cc8       ??_C@_0O@DMMHENKJ@cp_Descr_type@ 000000014001bcc8     bands.obj
 0002:00005cd8       ??_C@_0P@EEAFDJFH@cp_Field_class@ 000000014001bcd8     bands.obj
 0002:00005ce8       ??_C@_0O@FCFAPCDP@cp_Field_desc@ 000000014001bce8     bands.obj
 0002:00005cf8       ??_C@_0BA@LDOOFFKI@cp_Method_class@ 000000014001bcf8     bands.obj
 0002:00005d08       ??_C@_0P@NLGLFAKL@cp_Method_desc@ 000000014001bd08     bands.obj
 0002:00005d18       ??_C@_0BB@IIGJKIIK@cp_Imethod_class@ 000000014001bd18     bands.obj
 0002:00005d30       ??_C@_0BA@DCLGLKIL@cp_Imethod_desc@ 000000014001bd30     bands.obj
 0002:00005d40       ??_C@_0BI@NIJEEAN@cp_MethodHandle_refkind@ 000000014001bd40     bands.obj
 0002:00005d58       ??_C@_0BH@NKNCKAEO@cp_MethodHandle_member@ 000000014001bd58     bands.obj
 0002:00005d70       ??_C@_0O@NHPECHNH@cp_MethodType@ 000000014001bd70     bands.obj
 0002:00005d80       ??_C@_0BH@NPCIPIPL@cp_BootstrapMethod_ref@ 000000014001bd80     bands.obj
 0002:00005d98       ??_C@_0BN@DJLEBMBH@cp_BootstrapMethod_arg_count@ 000000014001bd98     bands.obj
 0002:00005db8       ??_C@_0BH@JNPGIEDO@cp_BootstrapMethod_arg@ 000000014001bdb8     bands.obj
 0002:00005dd0       ??_C@_0BG@CIPOMBAC@cp_InvokeDynamic_spec@ 000000014001bdd0     bands.obj
 0002:00005de8       ??_C@_0BG@IFFCPCPP@cp_InvokeDynamic_desc@ 000000014001bde8     bands.obj
 0002:00005e00       ??_C@_0BI@KJJNKCHD@attr_definition_headers@ 000000014001be00     bands.obj
 0002:00005e18       ??_C@_0BF@EEAHHHEA@attr_definition_name@ 000000014001be18     bands.obj
 0002:00005e30       ??_C@_0BH@EKDDDJNL@attr_definition_layout@ 000000014001be30     bands.obj
 0002:00005e48       ??_C@_0O@HJMNFDHJ@ic_this_class@ 000000014001be48     bands.obj
 0002:00005e58       ??_C@_08CKLAPDFF@ic_flags@ 000000014001be58     bands.obj
 0002:00005e68       ??_C@_0P@MGLGIOLC@ic_outer_class@ 000000014001be68     bands.obj
 0002:00005e78       ??_C@_07OPOCOJIH@ic_name@  000000014001be78     bands.obj
 0002:00005e80       ??_C@_0L@GONOGKKN@class_this@ 000000014001be80     bands.obj
 0002:00005e90       ??_C@_0M@FMPLOBH@class_super@ 000000014001be90     bands.obj
 0002:00005ea0       ??_C@_0BG@ELABOHHB@class_interface_count@ 000000014001bea0     bands.obj
 0002:00005eb8       ??_C@_0BA@GDKGLIFF@class_interface@ 000000014001beb8     bands.obj
 0002:00005ec8       ??_C@_0BC@GLACLOBG@class_field_count@ 000000014001bec8     bands.obj
 0002:00005ee0       ??_C@_0BD@MFLGOFPO@class_method_count@ 000000014001bee0     bands.obj
 0002:00005ef8       ??_C@_0M@IINMAGFA@field_descr@ 000000014001bef8     bands.obj
 0002:00005f08       ??_C@_0P@LDBPJHCP@field_flags_hi@ 000000014001bf08     bands.obj
 0002:00005f18       ??_C@_0P@OCEMJIHF@field_flags_lo@ 000000014001bf18     bands.obj
 0002:00005f28       ??_C@_0BB@GJGJJLKK@field_attr_count@ 000000014001bf28     bands.obj
 0002:00005f40       ??_C@_0BD@LLAABMND@field_attr_indexes@ 000000014001bf40     bands.obj
 0002:00005f58       ??_C@_0BB@LHINHPHH@field_attr_calls@ 000000014001bf58     bands.obj
 0002:00005f70       ??_C@_0BH@NKCAAIDC@field_ConstantValue_KQ@ 000000014001bf70     bands.obj
 0002:00005f88       ??_C@_0BD@HMEKDNDB@field_Signature_RS@ 000000014001bf88     bands.obj
 0002:00005fa0       ??_C@_0BF@KACJMLOM@field_metadata_bands@ 000000014001bfa0     bands.obj
 0002:00005fb8       ??_C@_0BB@NIMLDFOB@field_attr_bands@ 000000014001bfb8     bands.obj
 0002:00005fd0       ??_C@_0N@GLCNNANE@method_descr@ 000000014001bfd0     bands.obj
 0002:00005fe0       ??_C@_0BA@EIPLIEID@method_flags_hi@ 000000014001bfe0     bands.obj
 0002:00005ff0       ??_C@_0BA@BJKIILNJ@method_flags_lo@ 000000014001bff0     bands.obj
 0002:00006000       ??_C@_0BC@OPGFNCHF@method_attr_count@ 000000014001c000     bands.obj
 0002:00006018       ??_C@_0BE@LCKALKDL@method_attr_indexes@ 000000014001c018     bands.obj
 0002:00006030       ??_C@_0BC@DBIBDGKI@method_attr_calls@ 000000014001c030     bands.obj
 0002:00006048       ??_C@_0BE@HAIBKECN@method_Exceptions_N@ 000000014001c048     bands.obj
 0002:00006060       ??_C@_0BF@ILMHJLAD@method_Exceptions_RC@ 000000014001c060     bands.obj
 0002:00006078       ??_C@_0BE@HFOKJLNJ@method_Signature_RS@ 000000014001c078     bands.obj
 0002:00006090       ??_C@_0BG@JDLLNHF@method_metadata_bands@ 000000014001c090     bands.obj
 0002:000060a8       ??_C@_0BL@MNBFAABE@method_MethodParameters_NB@ 000000014001c0a8     bands.obj
 0002:000060c8       ??_C@_0CB@POGNKHAK@method_MethodParameters_name_RU@ 000000014001c0c8     bands.obj
 0002:000060f0       ??_C@_0CA@HDKLJONB@method_MethodParameters_flag_FH@ 000000014001c0f0     bands.obj
 0002:00006110       ??_C@_0BC@FOMHHMDO@method_attr_bands@ 000000014001c110     bands.obj
 0002:00006128       ??_C@_0P@DNMDIOJK@class_flags_hi@ 000000014001c128     bands.obj
 0002:00006138       ??_C@_0P@GMJAIBMA@class_flags_lo@ 000000014001c138     bands.obj
 0002:00006148       ??_C@_0BB@JELAOHEL@class_attr_count@ 000000014001c148     bands.obj
 0002:00006160       ??_C@_0BD@KFNGBOLA@class_attr_indexes@ 000000014001c160     bands.obj
 0002:00006178       ??_C@_0BB@EKFEADJG@class_attr_calls@ 000000014001c178     bands.obj
 0002:00006190       ??_C@_0BF@MJNFEGEM@class_SourceFile_RUN@ 000000014001c190     bands.obj
 0002:000061a8       ??_C@_0BJ@CCGEELON@class_EnclosingMethod_RC@ 000000014001c1a8     bands.obj
 0002:000061c8       ??_C@_0BK@LFCMIOIA@class_EnclosingMethod_RDN@ 000000014001c1c8     bands.obj
 0002:000061e8       ??_C@_0BD@GCJMDPFC@class_Signature_RS@ 000000014001c1e8     bands.obj
 0002:00006200       ??_C@_0BF@PHIMHC@class_metadata_bands@ 000000014001c200     bands.obj
 0002:00006218       ??_C@_0BF@PGJMDHG@class_InnerClasses_N@ 000000014001c218     bands.obj
 0002:00006230       ??_C@_0BG@HHABPLBI@class_InnerClasses_RC@ 000000014001c230     bands.obj
 0002:00006248       ??_C@_0BF@MHLAEJHO@class_InnerClasses_F@ 000000014001c248     bands.obj
 0002:00006260       ??_C@_0BN@FANFKEPF@class_InnerClasses_outer_RCN@ 000000014001c260     bands.obj
 0002:00006280       ??_C@_0BM@CHKHAMMI@class_InnerClasses_name_RUN@ 000000014001c280     bands.obj
 0002:000062a0       ??_C@_0CA@LBNJCLO@class_ClassFile_version_minor_H@ 000000014001c2a0     bands.obj
 0002:000062c0       ??_C@_0CA@KDGDJOMP@class_ClassFile_version_major_H@ 000000014001c2c0     bands.obj
 0002:000062e0       ??_C@_0BB@CFBCEJAA@class_attr_bands@ 000000014001c2e0     bands.obj
 0002:000062f8       ??_C@_0N@EJFJBMLJ@code_headers@ 000000014001c2f8     bands.obj
 0002:00006308       ??_C@_0P@DPBEANCA@code_max_stack@ 000000014001c308     bands.obj
 0002:00006318       ??_C@_0BD@OBGMDNFJ@code_max_na_locals@ 000000014001c318     bands.obj
 0002:00006330       ??_C@_0BD@OMMDBBC@code_handler_count@ 000000014001c330     bands.obj
 0002:00006348       ??_C@_0BF@NAEEIJON@code_handler_start_P@ 000000014001c348     bands.obj
 0002:00006360       ??_C@_0BE@GIJMHOG@code_handler_end_PO@ 000000014001c360     bands.obj
 0002:00006378       ??_C@_0BG@GJGNOMGM@code_handler_catch_PO@ 000000014001c378     bands.obj
 0002:00006390       ??_C@_0BH@ECFPKFHF@code_handler_class_RCN@ 000000014001c390     bands.obj
 0002:000063a8       ??_C@_0O@PKFJGJJN@code_flags_hi@ 000000014001c3a8     bands.obj
 0002:000063b8       ??_C@_0O@KLAKGGMH@code_flags_lo@ 000000014001c3b8     bands.obj
 0002:000063c8       ??_C@_0BA@OFJPMBMN@code_attr_count@ 000000014001c3c8     bands.obj
 0002:000063d8       ??_C@_0BC@BKACNFKP@code_attr_indexes@ 000000014001c3d8     bands.obj
 0002:000063f0       ??_C@_0BA@DLHLCFBA@code_attr_calls@ 000000014001c3f0     bands.obj
 0002:00006400       ??_C@_0BF@FNGGAIBD@code_StackMapTable_N@ 000000014001c400     bands.obj
 0002:00006418       ??_C@_0BL@IJLKAPMG@code_StackMapTable_frame_T@ 000000014001c418     bands.obj
 0002:00006438       ??_C@_0BL@FLGOBHFL@code_StackMapTable_local_N@ 000000014001c438     bands.obj
 0002:00006458       ??_C@_0BL@DBPDDGDK@code_StackMapTable_stack_N@ 000000014001c458     bands.obj
 0002:00006478       ??_C@_0BK@HMGLLHPP@code_StackMapTable_offset@ 000000014001c478     bands.obj
 0002:00006498       ??_C@_0BF@ONELPCMI@code_StackMapTable_T@ 000000014001c498     bands.obj
 0002:000064b0       ??_C@_0BG@EKILGBAE@code_StackMapTable_RC@ 000000014001c4b0     bands.obj
 0002:000064c8       ??_C@_0BF@IJCHDHMM@code_StackMapTable_P@ 000000014001c4c8     bands.obj
 0002:000064e0       ??_C@_0BH@EMJOIADC@code_LineNumberTable_N@ 000000014001c4e0     bands.obj
 0002:000064f8       ??_C@_0BL@BODGMFAF@code_LineNumberTable_bci_P@ 000000014001c4f8     bands.obj
 0002:00006518       ??_C@_0BK@KMDHKKJP@code_LineNumberTable_line@ 000000014001c518     bands.obj
 0002:00006538       ??_C@_0BK@EAEINMEG@code_LocalVariableTable_N@ 000000014001c538     bands.obj
 0002:00006558       ??_C@_0BO@EBBJALKI@code_LocalVariableTable_bci_P@ 000000014001c558     bands.obj
 0002:00006578       ??_C@_0BP@JIPNBFGM@code_LocalVariableTable_span_O@ 000000014001c578     bands.obj
 0002:00006598       ??_C@_0CA@LBKLALLO@code_LocalVariableTable_name_RU@ 000000014001c598     bands.obj
 0002:000065b8       ??_C@_0CA@OBPDECDH@code_LocalVariableTable_type_RS@ 000000014001c5b8     bands.obj
 0002:000065d8       ??_C@_0BN@BAELGOA@code_LocalVariableTable_slot@ 000000014001c5d8     bands.obj
 0002:000065f8       ??_C@_0BO@HHCIFDPC@code_LocalVariableTypeTable_N@ 000000014001c5f8     bands.obj
 0002:00006618       ??_C@_0CC@OECAEAHA@code_LocalVariableTypeTable_bci@ 000000014001c618     bands.obj
 0002:00006640       ??_C@_0CD@BAFAHGMB@code_LocalVariableTypeTable_spa@ 000000014001c640     bands.obj
 0002:00006668       ??_C@_0CE@BJEEHJII@code_LocalVariableTypeTable_nam@ 000000014001c668     bands.obj
 0002:00006690       ??_C@_0CE@EJBMDAAB@code_LocalVariableTypeTable_typ@ 000000014001c690     bands.obj
 0002:000066b8       ??_C@_0CB@DCPKAFMH@code_LocalVariableTypeTable_slo@ 000000014001c6b8     bands.obj
 0002:000066e0       ??_C@_0BA@FEDNGPIG@code_attr_bands@ 000000014001c6e0     bands.obj
 0002:000066f0       ??_C@_08ILNCKCLH@bc_codes@ 000000014001c6f0     bands.obj
 0002:00006700       ??_C@_0O@NHDHOKJ@bc_case_count@ 000000014001c700     bands.obj
 0002:00006710       ??_C@_0O@IPODCEHE@bc_case_value@ 000000014001c710     bands.obj
 0002:00006720       ??_C@_07PBCCPPFP@bc_byte@  000000014001c720     bands.obj
 0002:00006728       ??_C@_08LLANNIAP@bc_short@ 000000014001c728     bands.obj
 0002:00006738       ??_C@_08CNAAIOJJ@bc_local@ 000000014001c738     bands.obj
 0002:00006748       ??_C@_08CNIFPPEB@bc_label@ 000000014001c748     bands.obj
 0002:00006758       ??_C@_09LMIAJDCB@bc_intref@ 000000014001c758     bands.obj
 0002:00006768       ??_C@_0M@GHNOKACA@bc_floatref@ 000000014001c768     bands.obj
 0002:00006778       ??_C@_0L@FECALBEM@bc_longref@ 000000014001c778     bands.obj
 0002:00006788       ??_C@_0N@BLIIPDNE@bc_doubleref@ 000000014001c788     bands.obj
 0002:00006798       ??_C@_0N@MPKFBKGB@bc_stringref@ 000000014001c798     bands.obj
 0002:000067a8       ??_C@_0BE@JPNLPCGD@bc_loadablevalueref@ 000000014001c7a8     bands.obj
 0002:000067c0       ??_C@_0M@IBEIOBLC@bc_classref@ 000000014001c7c0     bands.obj
 0002:000067d0       ??_C@_0M@FHDAHFFG@bc_fieldref@ 000000014001c7d0     bands.obj
 0002:000067e0       ??_C@_0N@KBJNFGEO@bc_methodref@ 000000014001c7e0     bands.obj
 0002:000067f0       ??_C@_0O@BOILABNA@bc_imethodref@ 000000014001c7f0     bands.obj
 0002:00006800       ??_C@_0L@MEPMLOBJ@bc_indyref@ 000000014001c800     bands.obj
 0002:00006810       ??_C@_0N@CGLIFEKH@bc_thisfield@ 000000014001c810     bands.obj
 0002:00006820       ??_C@_0O@NMPFAKNK@bc_superfield@ 000000014001c820     bands.obj
 0002:00006830       ??_C@_0O@OCHHHCLJ@bc_thismethod@ 000000014001c830     bands.obj
 0002:00006840       ??_C@_0P@MMDJDCGG@bc_supermethod@ 000000014001c840     bands.obj
 0002:00006850       ??_C@_0L@IAPCGJHG@bc_initref@ 000000014001c850     bands.obj
 0002:00006860       ??_C@_09BGKIKDIC@bc_escref@ 000000014001c860     bands.obj
 0002:00006870       ??_C@_0O@LHNEEOML@bc_escrefsize@ 000000014001c870     bands.obj
 0002:00006880       ??_C@_0L@HJKABJFB@bc_escsize@ 000000014001c880     bands.obj
 0002:00006890       ??_C@_0L@HOKHNNPG@bc_escbyte@ 000000014001c890     bands.obj
 0002:000068a0       ??_C@_09GOEDCGAO@file_name@ 000000014001c8a0     bands.obj
 0002:000068b0       ??_C@_0N@INICLDFG@file_size_hi@ 000000014001c8b0     bands.obj
 0002:000068c0       ??_C@_0N@NMNBLMAM@file_size_lo@ 000000014001c8c0     bands.obj
 0002:000068d0       ??_C@_0N@JMABFCDG@file_modtime@ 000000014001c8d0     bands.obj
 0002:000068e0       ??_C@_0N@OPKBLMJG@file_options@ 000000014001c8e0     bands.obj
 0002:000068f0       ??_C@_08FPGGDHDD@no?5index@ 000000014001c8f0     bands.obj
 0002:00006900       ??_C@_08CHILEFNK@null?5ref@ 000000014001c900     bands.obj
 0002:00006910       ??_C@_07MLPLAPLE@bad?5ref@ 000000014001c910     bands.obj
 0002:00006918       ??_C@_0BC@CJBOIHCG@overflow?5detected@ 000000014001c918     bands.obj
 0002:00006930       ??_C@_0BJ@CALEAGEE@Native?5allocation?5failed@ 000000014001c930     bytes.obj
 0002:00006968       ??_C@_0BA@MMOCMGFH@bad?5value?5count@ 000000014001c968     coding.obj
 0002:00006978       ??_C@_0L@FLIJCFOD@bad?5coding@ 000000014001c978     coding.obj
 0002:00006988       ??_C@_0BE@IIPOPKNG@illegal?5arb?4?5coding@ 000000014001c988     coding.obj
 0002:000069a0       ??_C@_0BF@OEPDPLDN@illegal?5run?5encoding@ 000000014001c9a0     coding.obj
 0002:000069b8       ??_C@_0BM@FJMGNNPG@illegal?5nested?5run?5encoding@ 000000014001c9b8     coding.obj
 0002:000069d8       ??_C@_0BF@JOAAKECG@illegal?5pop?5encoding@ 000000014001c9d8     coding.obj
 0002:000069f0       ??_C@_0BM@CDDFICON@illegal?5nested?5pop?5encoding@ 000000014001c9f0     coding.obj
 0002:00006a10       ??_C@_0BG@HLIJPJNL@pop?4L?5value?5too?5small@ 000000014001ca10     coding.obj
 0002:00006a28       ??_C@_0BH@OCEIAIEJ@pop?5token?5out?5of?5range@ 000000014001ca28     coding.obj
 0002:00006a40       ??_C@_0CA@HBCNKKJO@bad?5meta?9coding?5for?5empty?5pop?1U@ 000000014001ca40     coding.obj
 0002:00006a60       ??_C@_0BA@DAENMACF@bad?5meta?9coding@ 000000014001ca60     coding.obj
 0002:00006a90       ??_C@_02DPKJAMEF@?$CFd@    000000014001ca90     main.obj
 0002:00006a98       ??_C@_09NIKIINED@unpack200@ 000000014001ca98     main.obj
 0002:00006aa8       ??_C@_0DM@OIAPDBBH@Usage?3?5?5?$CFs?5?$FL?9opt?4?4?4?5?$HM?5?9?9option?$DN@ 000000014001caa8     main.obj
 0002:00006af0       ??_C@_0CHL@BBGKGDMF@?6Unpacking?5Options?6?5?5?9H?$HLh?$HN?0?5?9?9d@ 000000014001caf0     main.obj
 0002:00006d70       ??_C@_0CJ@KKLFNMLF@?$CIFor?5more?5information?0?5run?5?$CFs?5?9@ 000000014001cd70     main.obj
 0002:00006da0       ??_C@_0BA@OCMGBEIP@UNPACK200_FLAGS@ 000000014001cda0     main.obj
 0002:00006db0       ??_C@_03CLFDNPKK@?6?7?5@   000000014001cdb0     main.obj
 0002:00006db8       ??_C@_0CB@HAIPLNAM@?9XDsuppress?9tool?9removal?9messag@ 000000014001cdb8     main.obj
 0002:00006de0       ??_C@_0P@BDFHEJH@Hdeflate?9hint?$DN@ 000000014001cde0     main.obj
 0002:00006df0       ??_C@_08KBJOIMAC@vverbose@ 000000014001cdf0     main.obj
 0002:00006dfc       ??_C@_06JKKBEHHF@qquiet@   000000014001cdfc     main.obj
 0002:00006e08       ??_C@_0BC@PMPEJJOP@rremove?9pack?9file@ 000000014001ce08     main.obj
 0002:00006e20       ??_C@_0L@ONHIOBCM@llog?9file?$DN@ 000000014001ce20     main.obj
 0002:00006e30       ??_C@_08KNEMGMJA@Vversion@ 000000014001ce30     main.obj
 0002:00006e3c       ??_C@_05GBNCKDGE@hhelp@    000000014001ce3c     main.obj
 0002:00006e50       ??_C@_0FL@LHNBJCPB@?6Warning?3?5The?5?$CFs?5tool?5is?5deprec@ 000000014001ce50     main.obj
 0002:00006eb0       ??_C@_0BE@DAFJFMML@unpack?4deflate?4hint@ 000000014001ceb0     main.obj
 0002:00006ec4       ??_C@_01HIHLOKLC@1@        000000014001cec4     main.obj
 0002:00006ec8       ??_C@_0DC@KGJOKPLE@com?4sun?4java?4util?4jar?4pack?4unpa@ 000000014001cec8     main.obj
 0002:00006f00       ??_C@_0P@BNKJLCIA@?$CFs?5version?5?$CFs?6@ 000000014001cf00     main.obj
 0002:00006f10       ??_C@_0BH@ODCNNNPJ@?5in?5$?$HLUNPACK200_FLAGS?$HN@ 000000014001cf10     main.obj
 0002:00006f28       ??_C@_0BN@OPJBPAAA@Missing?5option?5string?$CFs?3?5?$CFs?6@ 000000014001cf28     main.obj
 0002:00006f48       ??_C@_0BN@OCHJBIAD@Unrecognized?5argument?$CFs?3?5?$CFs?6@ 000000014001cf48     main.obj
 0002:00006f68       ??_C@_0CD@CEMFBAGC@com?4sun?4java?4util?4jar?4pack?4verb@ 000000014001cf68     main.obj
 0002:00006f90       ??_C@_0CL@JFLJFCLE@com?4sun?4java?4util?4jar?4pack?4unpa@ 000000014001cf90     main.obj
 0002:00006fc0       ??_C@_0BJ@LIHJOOPB@Unpacking?5from?5?$CFs?5to?5?$CFs?6@ 000000014001cfc0     main.obj
 0002:00006fdc       ??_C@_01JOAMLHOP@?9@       000000014001cfdc     main.obj
 0002:00006fe0       ??_C@_02JDPG@rb@           000000014001cfe0     main.obj
 0002:00006fe8       ??_C@_0CG@FKHOAOGE@Error?3?5Could?5not?5open?5input?5fil@ 000000014001cfe8     main.obj
 0002:00007010       ??_C@_0CC@NBFDMLEM@garbage?5after?5end?5of?5pack?5archi@ 000000014001d010     main.obj
 0002:00007038       ??_C@_0L@DCCGFMBN@Error?3?5?$CFs?6@ 000000014001d038     main.obj
 0002:00007048       ??_C@_0CD@KGGFLFGJ@unpacker?5completed?5with?5status?$DN@ 000000014001d048     main.obj
 0002:000070a8       ??_C@_0BC@DHBHLEDC@bad?5utf8?5encoding@ 000000014001d0a8     unpack.obj
 0002:000070c0       ??_C@_08MPEBFEBH@bad?5data@ 000000014001d0c0     unpack.obj
 0002:000070d0       ??_C@_0BI@MCADJHPK@missing?5class?5reference@ 000000014001d0d0     unpack.obj
 0002:000070e8       ??_C@_0BJ@DINDGABB@Internal?5buffer?5overflow@ 000000014001d0e8     unpack.obj
 0002:00007108       ??_C@_0BE@NBGJPKOJ@too?5much?5read?9ahead@ 000000014001d108     unpack.obj
 0002:00007120       ??_C@_0CB@MBENKFPE@EOF?5reading?5archive?5magic?5numbe@ 000000014001d120     unpack.obj
 0002:00007148       ??_C@_0M@HDHEHMIJ@Copy?9mode?4?6@ 000000014001d148     unpack.obj
 0002:00007160       ??_C@_0GN@MIAOKBBJ@?$EACorrupted?5pack?5file?3?5magic?1ver@ 000000014001d160     unpack.obj
 0002:000071d0       ??_C@_0DJ@EOFNCHGA@Format?5bits?5for?5Java?57?5must?5be?5@ 000000014001d1d0     unpack.obj
 0002:00007210       ??_C@_0DH@PDJEDCEA@High?5archive?5option?5bits?5are?5re@ 000000014001d210     unpack.obj
 0002:00007248       ??_C@_0BP@CKGMAJKP@EOF?5reading?5fixed?5input?5buffer@ 000000014001d248     unpack.obj
 0002:00007268       ??_C@_0BI@EDJMKDIH@impossible?5archive?5size@ 000000014001d268     unpack.obj
 0002:00007280       ??_C@_0DE@HNNKIDEL@cannot?5allocate?5large?5input?5buf@ 000000014001d280     unpack.obj
 0002:000072b8       ??_C@_0BL@KOJPDLNM@EOF?5reading?5archive?5header@ 000000014001d2b8     unpack.obj
 0002:000072d8       ??_C@_0BJ@HODOOMDO@EOF?5reading?5band?5headers@ 000000014001d2d8     unpack.obj
 0002:000072f8       ??_C@_0DD@FJENCPEO@A?5total?5of?5?$CFlld?5bytes?5were?5read@ 000000014001d2f8     unpack.obj
 0002:00007330       ??_C@_0DC@HIEHJDF@A?5total?5of?5?$CFlld?5file?5content?5by@ 000000014001d330     unpack.obj
 0002:00007370       ??_C@_0EH@BADKEGGH@A?5total?5of?5?$CFd?5files?5?$CIof?5which?5?$CF@ 000000014001d370     unpack.obj
 0002:000073b8       ??_C@_0DB@HCOAOCOI@archive?5too?5large?3?5?5constant?5po@ 000000014001d3b8     unpack.obj
 0002:000073f0       ??_C@_0BA@BMKLBFBL@bad?5utf8?5suffix@ 000000014001d3f0     unpack.obj
 0002:00007400       ??_C@_0BA@HHOGEFOO@bad?5utf8?5prefix@ 000000014001d400     unpack.obj
 0002:00007410       ??_C@_0BF@HNBIPEII@utf8?5prefix?5overflow@ 000000014001d410     unpack.obj
 0002:00007428       ??_C@_0BE@INMEHPDO@unexpected?5band?5?$CFs?6@ 000000014001d428     unpack.obj
 0002:00007440       ??_C@_0BKA@JMJPKLFN@01?$AASignature?$AADeprecated?$AARuntime@ 000000014001d440     unpack.obj
 0002:000075e0       ??_C@_0BK@NOGBJPAL@attribute?5index?5too?5large@ 000000014001d5e0     unpack.obj
 0002:00007600       ??_C@_0BK@OFNJKMED@redefined?5attribute?5index@ 000000014001d600     unpack.obj
 0002:00007620       ??_C@_0BJ@OGDEGNBN@garbage?5at?5end?5of?5layout@ 000000014001d620     unpack.obj
 0002:00007640       ??_C@_0BN@NJCEKHIO@garbage?5mixed?5with?5callables@ 000000014001d640     unpack.obj
 0002:00007660       ??_C@_0BD@BJONMNHI@bad?5call?5in?5layout@ 000000014001d660     unpack.obj
 0002:00007678       ??_C@_0BD@EOHIHJFP@bad?5layout?5element@ 000000014001d678     unpack.obj
 0002:00007690       ??_C@_0BK@CHPLBKBJ@missing?5numeral?5in?5layout@ 000000014001d690     unpack.obj
 0002:000076b0       ??_C@_0BB@FJJKEHGJ@numeral?5overflow@ 000000014001d6b0     unpack.obj
 0002:000076c8       ??_C@_0P@HDHNKEAB@bad?5union?5case@ 000000014001d6c8     unpack.obj
 0002:000076d8       ??_C@_0DD@PGOJPNFL@bad?5range?5in?5union?5case?5label?5?$CI@ 000000014001d6d8     unpack.obj
 0002:00007710       ??_C@_0BO@JELFCPB@bad?5range?5in?5union?5case?5label@ 000000014001d710     unpack.obj
 0002:00007730       ??_C@_0P@KBKJHJBF@bad?5case?5label@ 000000014001d730     unpack.obj
 0002:00007740       ??_C@_0P@MNJPOPJO@bad?5call?5label@ 000000014001d740     unpack.obj
 0002:00007750       ??_C@_0BF@ILAEDGAO@bad?5reference?5layout@ 000000014001d750     unpack.obj
 0002:00007768       ??_C@_0BE@NGGDBALG@bad?5nested?5callable@ 000000014001d768     unpack.obj
 0002:00007780       ??_C@_0L@FLEMDFJG@bad?5layout@ 000000014001d780     unpack.obj
 0002:00007790       ??_C@_0JK@BMMFGJDP@?$FLNB?$FL?$CI1?$CJ?$FN?$FN?$FLNH?$FL?$CI1?$CJ?$FN?$FN?$FLRSHNH?$FLRUH?$CI1?$CJ@ 000000014001d790     unpack.obj
 0002:00007830       ??_C@_09MAEOCCFN@?$FLNB?$FL?$CI1?$CJ?$FN?$FN@ 000000014001d830     unpack.obj
 0002:00007840       ??_C@_0CC@PCCOCALL@?$FLNB?$FL?$CI1?$CJ?$FN?$FN?$FLNH?$FL?$CI1?$CJ?$FN?$FN?$FLRSHNH?$FLRUH?$CI1?$CJ@ 000000014001d840     unpack.obj
 0002:00007870       ??_C@_0BBL@GCIMMLOG@?$FLNH?$FL?$CI1?$CJ?$CI2?$CJ?$CI3?$CJ?$FN?$FN?$FLTB?$CI0?01?$CJ?$FLB?$FN?$CI16?$CJ?$FL@ 000000014001d870     unpack.obj
 0002:00007990       ??_C@_0BK@CIMGHPDJ@RuntimeVisibleAnnotations@ 000000014001d990     unpack.obj
 0002:000079b0       ??_C@_0BM@BNNGFNMF@RuntimeInvisibleAnnotations@ 000000014001d9b0     unpack.obj
 0002:000079d0       ??_C@_0CD@ONLIBICP@RuntimeVisibleParameterAnnotati@ 000000014001d9d0     unpack.obj
 0002:000079f8       ??_C@_0CF@BFEAEHFK@RuntimeInvisibleParameterAnnota@ 000000014001d9f8     unpack.obj
 0002:00007a20       ??_C@_0BC@DAGIEPHG@AnnotationDefault@ 000000014001da20     unpack.obj
 0002:00007a38       ??_C@_0BO@IJLELCEA@RuntimeVisibleTypeAnnotations@ 000000014001da38     unpack.obj
 0002:00007a58       ??_C@_0CA@GCLMFPKD@RuntimeInvisibleTypeAnnotations@ 000000014001da58     unpack.obj
 0002:00007a78       ??_C@_0BG@FDJMCAOP@identical?5inner?5class@ 000000014001da78     unpack.obj
 0002:00007a90       ??_C@_0BN@GFADPNEE@undefined?5attribute?5flag?5bit@ 000000014001da90     unpack.obj
 0002:00007ab0       ??_C@_0BO@CMGKNLIA@attribute?5index?5out?5of?5bounds@ 000000014001dab0     unpack.obj
 0002:00007ad0       ??_C@_0DH@OHIKFIJI@undefined?5StackMapTable?5attribu@ 000000014001dad0     unpack.obj
 0002:00007b08       ??_C@_0CL@CLGKHLIF@layout_definition?5pointer?5must?5@ 000000014001db08     unpack.obj
 0002:00007b38       ??_C@_0CE@NENNCDNJ@putlayout?3?5unexpected?5NULL?5for?5@ 000000014001db38     unpack.obj
 0002:00007b60       ??_C@_0BB@HNCAJEIE@cp?5utf8?5overflow@ 000000014001db60     unpack.obj
 0002:00007b78       ??_C@_0BC@IJJDHGHN@cp?5class?5overflow@ 000000014001db78     unpack.obj
 0002:00007b90       ??_C@_0DE@FNJPLIMN@com?4sun?4java?4util?4jar?4pack?4unpa@ 000000014001db90     unpack.obj
 0002:00007bc4       ??_C@_04LKOEDJLC@keep@     000000014001dbc4     unpack.obj
 0002:00007bd0       ??_C@_0CJ@LFNCLCEP@com?4sun?4java?4util?4jar?4pack?4verb@ 000000014001dbd0     unpack.obj
 0002:00007bfc       ??_C@_03CGLHMDPP@now@      000000014001dbfc     unpack.obj
 0002:00007c00       ??_C@_0DL@GFEANCIP@After?5segment?5?$CFd?0?5?$CFlld?5bytes?5re@ 000000014001dc00     unpack.obj
 0002:00007c40       ??_C@_0EJ@CMEPGJEN@After?5segment?5?$CFd?0?5?$CFd?5files?5?$CIof?5@ 000000014001dc40     unpack.obj
 0002:00007c8c       ??_C@_01LKDEMHDF@s@        000000014001dc8c     unpack.obj
 0002:00007c90       ??_C@_0DH@GNBHDKCB@After?5segment?5?$CFd?0?5?$CFd?5segment?$CFs?5@ 000000014001dc90     unpack.obj
 0002:00007cc8       ??_C@_09GHCKAPML@?$CInot?5set?$CJ@ 000000014001dcc8     unpack.obj
 0002:00007cd4       ??_C@_06BAKFFEGN@?$CFs?$DN?$CFs?6@ 000000014001dcd4     unpack.obj
 0002:00007ce0       ??_C@_0BB@MNFIFPBF@bad?5KQ?5reference@ 000000014001dce0     unpack.obj
 0002:00007cf8       ??_C@_0L@PDBBHOGB@bad?5bcimap@ 000000014001dcf8     unpack.obj
 0002:00007d08       ??_C@_0BM@GPDDEOEP@too?5many?5InnerClasses?5attrs@ 000000014001dd08     unpack.obj
 0002:00007d24       ??_C@_05PBJILJE@?4java@    000000014001dd24     unpack.obj
 0002:00007d30       ??_C@_0BB@MICPNADP@bad?5layout?5index@ 000000014001dd30     unpack.obj
 0002:00007d48       ??_C@_0BE@BKLBLMJK@bad?5attribute?5index@ 000000014001dd48     unpack.obj
 0002:00007d60       ??_C@_0BN@CLDGGNCI@bad?5reference?5to?5inner?5class@ 000000014001dd60     unpack.obj
 0002:00007d80       ??_C@_0P@DHEBFDOP@Internal?5error@ 000000014001dd80     unpack.obj
 0002:00007d90       ??_C@_0CC@IOEIADGN@archive?5header?5had?5incorrect?5si@ 000000014001dd90     unpack.obj
 0002:00007db8       ??_C@_0BM@NDDMOHPH@class?5file?5size?5transmitted@ 000000014001ddb8     unpack.obj
 0002:00007dd4       ??_C@_06POIMOJKC@?4class@  000000014001ddd4     unpack.obj
 0002:00007de0       ??_C@_0BK@NJPACPAH@EOF?5reading?5resource?5file@ 000000014001dde0     unpack.obj
 0002:00007e00       ??_C@_0BJ@NEMIFNOC@Wrote?5?$CFlld?5bytes?5to?3?5?$CFs?6@ 000000014001de00     unpack.obj
 0002:00007e1c       ??_C@_02DPNLHKJD@a?$CL@    000000014001de1c     unpack.obj
 0002:00007e20       ??_C@_0BK@NDLGHGBM@Can?5not?5open?5log?5file?5?$CFs?6@ 000000014001de20     unpack.obj
 0002:00007e40       ??_C@_0BI@CELHNJPG@error?5unpacking?5archive@ 000000014001de40     unpack.obj
 0002:00007e58       ??_C@_03OFAPEBGM@?$CFs?6@  000000014001de58     unpack.obj
 0002:00007e60       __xmm@00000000000000ab00000001000000aa 000000014001de60     unpack.obj
 0002:00007e70       __xmm@00000001000000a00000000700000096 000000014001de70     unpack.obj
 0002:00007e80       ??_C@_0CE@HLJAOJEP@corrupt?5pack?5file?5or?5internal?5e@ 000000014001de80     utils.obj
 0002:00007ea8       ??_C@_0BF@JFFKOPFD@Error?3?5unpacker?3?5?$CFs?6@ 000000014001dea8     utils.obj
 0002:00007ec0       ??_C@_0CG@HFNCMKIN@Error?3?5unpacker?3?5no?5current?5ins@ 000000014001dec0     utils.obj
 0002:00007ef8       ??_C@_0CL@EKHPJDGB@Error?3?5write?5on?5output?5file?5fai@ 000000014001def8     zip.obj
 0002:00007f24       ??_C@_02GMLFBBN@wb@        000000014001df24     zip.obj
 0002:00007f28       ??_C@_0CE@COMJCOPK@Error?3?5Could?5not?5open?5jar?5file?3@ 000000014001df28     zip.obj
 0002:00007f50       ??_C@_0CO@DCPNMPAF@Error?3?5gmtime?5failure?0?5invalid?5@ 000000014001df50     zip.obj
 0002:00007f80       ??_C@_0BG@NMMFCDCO@error?5inflating?5input@ 000000014001df80     zip.obj
 0002:00007f98       ??_C@_0CL@NMECEKOA@garbage?5after?5end?5of?5deflated?5i@ 000000014001df98     zip.obj
 0002:00007fc8       ??_C@_0DL@PJJNLKFP@Error?3reading?5CRC?5information?5o@ 000000014001dfc8     zip.obj
 0002:00008008       ??_C@_0DH@LPFNBMGH@Error?3reading?5file?5length?5on?5in@ 000000014001e008     zip.obj
 0002:00008040       ??_C@_0CE@EBLNOIJH@CRC?5error?0?5invalid?5compressed?5d@ 000000014001e040     zip.obj
 0002:00008068       ??_C@_0BE@BDJJEDBE@cannot?5create?5input@ 000000014001e068     zip.obj
 0002:00008080       ??_C@_0BE@BMGPHILO@short?5stream?5header@ 000000014001e080     zip.obj
 0002:000080b0       __xmm@ffffffffffffffffffffffffffffffff 000000014001e0b0     MSVCRT:utility.obj
 0002:000080c0       _load_config_used          000000014001e0c0     MSVCRT:loadcfg.obj
 0002:00008280       __volatile_metadata        000000014001e280     <linker-defined>
 0002:000085d8       __rtc_iaa                  000000014001e5d8     MSVCRT:initsect.obj
 0002:000085e0       __rtc_izz                  000000014001e5e0     MSVCRT:initsect.obj
 0002:000085e8       __rtc_taa                  000000014001e5e8     MSVCRT:initsect.obj
 0002:000085f0       __rtc_tzz                  000000014001e5f0     MSVCRT:initsect.obj
 0002:00008e48       __IMPORT_DESCRIPTOR_KERNEL32 000000014001ee48     kernel32:KERNEL32.dll
 0002:00008e5c       __IMPORT_DESCRIPTOR_VCRUNTIME140 000000014001ee5c     vcruntime:VCRUNTIME140.dll
 0002:00008e70       __IMPORT_DESCRIPTOR_api-ms-win-crt-heap-l1-1-0 000000014001ee70     ucrt:api-ms-win-crt-heap-l1-1-0.dll
 0002:00008e84       __IMPORT_DESCRIPTOR_api-ms-win-crt-stdio-l1-1-0 000000014001ee84     ucrt:api-ms-win-crt-stdio-l1-1-0.dll
 0002:00008e98       __IMPORT_DESCRIPTOR_api-ms-win-crt-filesystem-l1-1-0 000000014001ee98     ucrt:api-ms-win-crt-filesystem-l1-1-0.dll
 0002:00008eac       __IMPORT_DESCRIPTOR_api-ms-win-crt-runtime-l1-1-0 000000014001eeac     ucrt:api-ms-win-crt-runtime-l1-1-0.dll
 0002:00008ec0       __IMPORT_DESCRIPTOR_api-ms-win-crt-string-l1-1-0 000000014001eec0     ucrt:api-ms-win-crt-string-l1-1-0.dll
 0002:00008ed4       __IMPORT_DESCRIPTOR_api-ms-win-crt-environment-l1-1-0 000000014001eed4     ucrt:api-ms-win-crt-environment-l1-1-0.dll
 0002:00008ee8       __IMPORT_DESCRIPTOR_api-ms-win-crt-utility-l1-1-0 000000014001eee8     ucrt:api-ms-win-crt-utility-l1-1-0.dll
 0002:00008efc       __IMPORT_DESCRIPTOR_api-ms-win-crt-convert-l1-1-0 000000014001eefc     ucrt:api-ms-win-crt-convert-l1-1-0.dll
 0002:00008f10       __IMPORT_DESCRIPTOR_api-ms-win-crt-time-l1-1-0 000000014001ef10     ucrt:api-ms-win-crt-time-l1-1-0.dll
 0002:00008f24       __IMPORT_DESCRIPTOR_api-ms-win-crt-math-l1-1-0 000000014001ef24     ucrt:api-ms-win-crt-math-l1-1-0.dll
 0002:00008f38       __IMPORT_DESCRIPTOR_api-ms-win-crt-locale-l1-1-0 000000014001ef38     ucrt:api-ms-win-crt-locale-l1-1-0.dll
 0002:00008f4c       __NULL_IMPORT_DESCRIPTOR   000000014001ef4c     kernel32:KERNEL32.dll
 0003:00000000       ?basic_codings@@3PAUcoding@@A 0000000140020000     coding.obj
 0003:00000b70       __security_cookie_complement 0000000140020b70     MSVCRT:gs_cookie.obj
 0003:00000b78       __security_cookie          0000000140020b78     MSVCRT:gs_cookie.obj
 0003:00000b80       __scrt_native_dllmain_reason 0000000140020b80     MSVCRT:utility.obj
 0003:00000b84       __scrt_default_matherr     0000000140020b84     MSVCRT:matherr.obj
 0003:00000b88       __isa_available            0000000140020b88     MSVCRT:cpu_disp.obj
 0003:00000b8c       __isa_enabled              0000000140020b8c     MSVCRT:cpu_disp.obj
 0003:00000b90       __memset_fast_string_threshold 0000000140020b90     MSVCRT:cpu_disp.obj
 0003:00000b98       __memset_nt_threshold      0000000140020b98     MSVCRT:cpu_disp.obj
 0003:00000ba0       __scrt_ucrt_dll_is_in_use  0000000140020ba0     MSVCRT:ucrt_stubs.obj
 0003:00000fb8       ?non_mt_current@unpacker@@2PEAU1@EA 0000000140020fb8     main.obj
 0003:00000fc8       ?_OptionsStorage@?1??__local_stdio_printf_options@@9@4_KA 0000000140020fc8     main.obj
 0003:00001550       __scrt_current_native_startup_state 0000000140021550     MSVCRT:utility.obj
 0003:00001558       __scrt_native_startup_lock 0000000140021558     MSVCRT:utility.obj
 0003:000015a0       ?__type_info_root_node@@3U__type_info_node@@A 00000001400215a0     MSVCRT:tncleanup.obj
 0003:000015b0       ?_OptionsStorage@?1??__local_stdio_scanf_options@@9@4_KA 00000001400215b0     MSVCRT:default_local_stdio_options.obj
 0003:000015b8       __scrt_debugger_hook_flag  00000001400215b8     MSVCRT:utility_desktop.obj
 0003:000015bc       __favor                    00000001400215bc     MSVCRT:cpu_disp.obj
 0003:000015c0       __dyn_tls_dtor_callback    00000001400215c0     <common>
 0003:000015c8       __dyn_tls_init_callback    00000001400215c8     <common>

 entry point at        0001:000140a0

 Static symbols

 0000:fffdb000       .debug$S                   0000000140000000     unpack200.exp
 0000:fffdb000       .debug$S                   0000000140000000     vcruntime:VCRUNTIME140.dll
 0000:fffdb000       .debug$S                   0000000140000000     vcruntime:VCRUNTIME140.dll
 0000:fffdb000       .debug$S                   0000000140000000     vcruntime:VCRUNTIME140.dll
 0000:fffdb000       .debug$S                   0000000140000000     vcruntime:VCRUNTIME140.dll
 0000:fffdb000       .debug$S                   0000000140000000     vcruntime:VCRUNTIME140.dll
 0000:fffdb000       .debug$S                   0000000140000000     vcruntime:VCRUNTIME140.dll
 0000:fffdb000       .debug$S                   0000000140000000     vcruntime:VCRUNTIME140.dll
 0000:fffdb000       .debug$S                   0000000140000000     vcruntime:VCRUNTIME140.dll
 0000:fffdb000       .debug$S                   0000000140000000     vcruntime:VCRUNTIME140.dll
 0000:fffdb000       .debug$S                   0000000140000000     vcruntime:VCRUNTIME140.dll
 0000:fffdb000       .debug$S                   0000000140000000     ucrt:api-ms-win-crt-convert-l1-1-0.dll
 0000:fffdb000       .debug$S                   0000000140000000     ucrt:api-ms-win-crt-environment-l1-1-0.dll
 0000:fffdb000       .debug$S                   0000000140000000     ucrt:api-ms-win-crt-filesystem-l1-1-0.dll
 0000:fffdb000       .debug$S                   0000000140000000     ucrt:api-ms-win-crt-filesystem-l1-1-0.dll
 0000:fffdb000       .debug$S                   0000000140000000     ucrt:api-ms-win-crt-heap-l1-1-0.dll
 0000:fffdb000       .debug$S                   0000000140000000     ucrt:api-ms-win-crt-heap-l1-1-0.dll
 0000:fffdb000       .debug$S                   0000000140000000     ucrt:api-ms-win-crt-heap-l1-1-0.dll
 0000:fffdb000       .debug$S                   0000000140000000     ucrt:api-ms-win-crt-heap-l1-1-0.dll
 0000:fffdb000       .debug$S                   0000000140000000     ucrt:api-ms-win-crt-heap-l1-1-0.dll
 0000:fffdb000       .debug$S                   0000000140000000     ucrt:api-ms-win-crt-locale-l1-1-0.dll
 0000:fffdb000       .debug$S                   0000000140000000     ucrt:api-ms-win-crt-math-l1-1-0.dll
 0000:fffdb000       .debug$S                   0000000140000000     ucrt:api-ms-win-crt-runtime-l1-1-0.dll
 0000:fffdb000       .debug$S                   0000000140000000     ucrt:api-ms-win-crt-runtime-l1-1-0.dll
 0000:fffdb000       .debug$S                   0000000140000000     ucrt:api-ms-win-crt-runtime-l1-1-0.dll
 0000:fffdb000       .debug$S                   0000000140000000     ucrt:api-ms-win-crt-runtime-l1-1-0.dll
 0000:fffdb000       .debug$S                   0000000140000000     ucrt:api-ms-win-crt-runtime-l1-1-0.dll
 0000:fffdb000       .debug$S                   0000000140000000     ucrt:api-ms-win-crt-runtime-l1-1-0.dll
 0000:fffdb000       .debug$S                   0000000140000000     ucrt:api-ms-win-crt-runtime-l1-1-0.dll
 0000:fffdb000       .debug$S                   0000000140000000     ucrt:api-ms-win-crt-runtime-l1-1-0.dll
 0000:fffdb000       .debug$S                   0000000140000000     ucrt:api-ms-win-crt-runtime-l1-1-0.dll
 0000:fffdb000       .debug$S                   0000000140000000     ucrt:api-ms-win-crt-runtime-l1-1-0.dll
 0000:fffdb000       .debug$S                   0000000140000000     ucrt:api-ms-win-crt-runtime-l1-1-0.dll
 0000:fffdb000       .debug$S                   0000000140000000     ucrt:api-ms-win-crt-runtime-l1-1-0.dll
 0000:fffdb000       .debug$S                   0000000140000000     ucrt:api-ms-win-crt-runtime-l1-1-0.dll
 0000:fffdb000       .debug$S                   0000000140000000     ucrt:api-ms-win-crt-runtime-l1-1-0.dll
 0000:fffdb000       .debug$S                   0000000140000000     ucrt:api-ms-win-crt-runtime-l1-1-0.dll
 0000:fffdb000       .debug$S                   0000000140000000     ucrt:api-ms-win-crt-runtime-l1-1-0.dll
 0000:fffdb000       .debug$S                   0000000140000000     ucrt:api-ms-win-crt-runtime-l1-1-0.dll
 0000:fffdb000       .debug$S                   0000000140000000     ucrt:api-ms-win-crt-runtime-l1-1-0.dll
 0000:fffdb000       .debug$S                   0000000140000000     ucrt:api-ms-win-crt-runtime-l1-1-0.dll
 0000:fffdb000       .debug$S                   0000000140000000     ucrt:api-ms-win-crt-runtime-l1-1-0.dll
 0000:fffdb000       .debug$S                   0000000140000000     ucrt:api-ms-win-crt-runtime-l1-1-0.dll
 0000:fffdb000       .debug$S                   0000000140000000     ucrt:api-ms-win-crt-runtime-l1-1-0.dll
 0000:fffdb000       .debug$S                   0000000140000000     ucrt:api-ms-win-crt-runtime-l1-1-0.dll
 0000:fffdb000       .debug$S                   0000000140000000     ucrt:api-ms-win-crt-stdio-l1-1-0.dll
 0000:fffdb000       .debug$S                   0000000140000000     ucrt:api-ms-win-crt-stdio-l1-1-0.dll
 0000:fffdb000       .debug$S                   0000000140000000     ucrt:api-ms-win-crt-stdio-l1-1-0.dll
 0000:fffdb000       .debug$S                   0000000140000000     ucrt:api-ms-win-crt-stdio-l1-1-0.dll
 0000:fffdb000       .debug$S                   0000000140000000     ucrt:api-ms-win-crt-stdio-l1-1-0.dll
 0000:fffdb000       .debug$S                   0000000140000000     ucrt:api-ms-win-crt-stdio-l1-1-0.dll
 0000:fffdb000       .debug$S                   0000000140000000     ucrt:api-ms-win-crt-stdio-l1-1-0.dll
 0000:fffdb000       .debug$S                   0000000140000000     ucrt:api-ms-win-crt-stdio-l1-1-0.dll
 0000:fffdb000       .debug$S                   0000000140000000     ucrt:api-ms-win-crt-stdio-l1-1-0.dll
 0000:fffdb000       .debug$S                   0000000140000000     ucrt:api-ms-win-crt-stdio-l1-1-0.dll
 0000:fffdb000       .debug$S                   0000000140000000     ucrt:api-ms-win-crt-stdio-l1-1-0.dll
 0000:fffdb000       .debug$S                   0000000140000000     ucrt:api-ms-win-crt-stdio-l1-1-0.dll
 0000:fffdb000       .debug$S                   0000000140000000     ucrt:api-ms-win-crt-string-l1-1-0.dll
 0000:fffdb000       .debug$S                   0000000140000000     ucrt:api-ms-win-crt-string-l1-1-0.dll
 0000:fffdb000       .debug$S                   0000000140000000     ucrt:api-ms-win-crt-string-l1-1-0.dll
 0000:fffdb000       .debug$S                   0000000140000000     ucrt:api-ms-win-crt-string-l1-1-0.dll
 0000:fffdb000       .debug$S                   0000000140000000     ucrt:api-ms-win-crt-string-l1-1-0.dll
 0000:fffdb000       .debug$S                   0000000140000000     ucrt:api-ms-win-crt-string-l1-1-0.dll
 0000:fffdb000       .debug$S                   0000000140000000     ucrt:api-ms-win-crt-string-l1-1-0.dll
 0000:fffdb000       .debug$S                   0000000140000000     ucrt:api-ms-win-crt-string-l1-1-0.dll
 0000:fffdb000       .debug$S                   0000000140000000     ucrt:api-ms-win-crt-time-l1-1-0.dll
 0000:fffdb000       .debug$S                   0000000140000000     ucrt:api-ms-win-crt-time-l1-1-0.dll
 0000:fffdb000       .debug$S                   0000000140000000     ucrt:api-ms-win-crt-utility-l1-1-0.dll
 0000:fffdb000       .debug$S                   0000000140000000     kernel32:KERNEL32.dll
 0000:fffdb000       .debug$S                   0000000140000000     kernel32:KERNEL32.dll
 0000:fffdb000       .debug$S                   0000000140000000     kernel32:KERNEL32.dll
 0000:fffdb000       .debug$S                   0000000140000000     kernel32:KERNEL32.dll
 0000:fffdb000       .debug$S                   0000000140000000     kernel32:KERNEL32.dll
 0000:fffdb000       .debug$S                   0000000140000000     kernel32:KERNEL32.dll
 0000:fffdb000       .debug$S                   0000000140000000     kernel32:KERNEL32.dll
 0000:fffdb000       .debug$S                   0000000140000000     kernel32:KERNEL32.dll
 0000:fffdb000       .debug$S                   0000000140000000     kernel32:KERNEL32.dll
 0000:fffdb000       .debug$S                   0000000140000000     kernel32:KERNEL32.dll
 0000:fffdb000       .debug$S                   0000000140000000     kernel32:KERNEL32.dll
 0000:fffdb000       .debug$S                   0000000140000000     kernel32:KERNEL32.dll
 0000:fffdb000       .debug$S                   0000000140000000     kernel32:KERNEL32.dll
 0000:fffdb000       .debug$S                   0000000140000000     kernel32:KERNEL32.dll
 0000:fffdb000       .debug$S                   0000000140000000     kernel32:KERNEL32.dll
 0000:fffdb000       .debug$S                   0000000140000000     kernel32:KERNEL32.dll
 0001:00000000       deflate_stored             0000000140001000 f   deflate.obj
 0001:00000424       deflate_fast               0000000140001424 f   deflate.obj
 0001:00000860       deflate_slow               0000000140001860 f   deflate.obj
 0001:00001b98       deflateStateCheck          0000000140002b98 f   deflate.obj
 0001:00001bec       deflate_huff               0000000140002bec f   deflate.obj
 0001:00001db8       deflate_rle                0000000140002db8 f   deflate.obj
 0001:00002104       fill_window                0000000140003104 f   deflate.obj
 0001:0000230c       flush_pending              000000014000330c f   deflate.obj
 0001:00002380       lm_init                    0000000140003380 f   deflate.obj
 0001:0000242c       longest_match              000000014000342c f   deflate.obj
 0001:000025dc       read_buf                   00000001400035dc f   deflate.obj
 0001:00002670       slide_hash                 0000000140003670 f   deflate.obj
 0001:00004070       $LN790                     0000000140005070     inflate.obj
 0001:00004370       inflateStateCheck          0000000140005370 f   inflate.obj
 0001:000043a8       updatewindow               00000001400053a8 f   inflate.obj
 0001:00004ec4       bi_flush                   0000000140005ec4 f   trees.obj
 0001:00004f3c       bi_windup                  0000000140005f3c f   trees.obj
 0001:00004f94       build_tree                 0000000140005f94 f   trees.obj
 0001:0000524c       compress_block             000000014000624c f   trees.obj
 0001:000056a4       gen_bitlen                 00000001400066a4 f   trees.obj
 0001:000058c0       init_block                 00000001400068c0 f   trees.obj
 0001:00005930       pqdownheap                 0000000140006930 f   trees.obj
 0001:000059e4       scan_tree                  00000001400069e4 f   trees.obj
 0001:00005af8       send_all_trees             0000000140006af8 f   trees.obj
 0001:00005d88       send_tree                  0000000140006d88 f   trees.obj
 0001:0000833c       ?nbasename@@YAPEBDPEBD@Z   000000014000933c f   main.obj
 0001:00008364       ?read_input_via_stdio@@YA_JPEAUunpacker@@PEAX_J2@Z 0000000140009364 f   main.obj
 0001:00008408       ?read_magic@@YAHPEAUunpacker@@QEADH@Z 0000000140009408 f   main.obj
 0001:00008c6c       ?usage@@YAXPEAUunpacker@@PEBD_N@Z 0000000140009c6c f   main.obj
 0001:00009188       ?compare_Utf8_chars@@YAHAEAUbytes@@0@Z 000000014000a188 f   unpack.obj
 0001:00010230       ?store_Utf8_char@@YAPEACPEACG@Z 0000000140011230 f   unpack.obj
 0001:00013344       ?read_input_via_gzip@@YA_JPEAUunpacker@@PEAX_J2@Z 0000000140014344 f   zip.obj
 0001:00013c44       capture_current_context    0000000140014c44 f   MSVCRT:gs_report.obj
 0001:00013cb4       capture_previous_context   0000000140014cb4 f   MSVCRT:gs_report.obj
 0001:00013db0       $$000000                   0000000140014db0     MSVCRT:amdsecgs.obj
 0001:00013de0       $$000000                   0000000140014de0     MSVCRT:chkstk.obj
 0001:00013e40       ?pre_c_initialization@@YAHXZ 0000000140014e40 f   MSVCRT:exe_main.obj
 0001:00013ef8       ?post_pgo_initialization@@YAHXZ 0000000140014ef8 f   MSVCRT:exe_main.obj
 0001:00013f08       ?pre_cpp_initialization@@YAXXZ 0000000140014f08 f   MSVCRT:exe_main.obj
 0001:00013f24       ?__scrt_common_main_seh@@YAHXZ 0000000140014f24 f   MSVCRT:exe_main.obj
 0001:00014940       $$000000                   0000000140015940     MSVCRT:guard_dispatch.obj
 0001:00014960       $$000000                   0000000140015960     MSVCRT:guard_xfg_dispatch.obj
 0001:00014976       ?filt$0@?0??__scrt_common_main_seh@@YAHXZ@4HA 0000000140015976 f   MSVCRT:exe_main.obj
 0001:00014994       __scrt_is_nonwritable_in_current_image$filt$0 0000000140015994 f   MSVCRT:utility.obj
 0002:00000300       ?pre_cpp_initializer@@3P6AXXZEA 0000000140016300     MSVCRT:exe_main.obj
 0002:00000318       ?pre_c_initializer@@3P6AHXZEA 0000000140016318     MSVCRT:exe_main.obj
 0002:00000320       ?post_pgo_initializer@@3P6AHXZEA 0000000140016320     MSVCRT:exe_main.obj
 0002:000003a4       ?my_version@?1??deflateInit2_@@9@9 00000001400163a4     deflate.obj
 0002:000003b0       configuration_table        00000001400163b0     deflate.obj
 0002:00000450       ?lenfix@?1??fixedtables@@9@9 0000000140016450     infback.obj
 0002:00000c50       ?distfix@?1??fixedtables@@9@9 0000000140016c50     infback.obj
 0002:00000cd0       ?order@?1??inflateBack@@9@9 0000000140016cd0     infback.obj
 0002:00000e50       ?lenfix@?1??fixedtables@@9@9 0000000140016e50     inflate.obj
 0002:00001650       ?distfix@?1??fixedtables@@9@9 0000000140017650     inflate.obj
 0002:000016d0       ?order@?1??inflate@@9@9    00000001400176d0     inflate.obj
 0002:000017e0       ?lbase@?1??inflate_table@@9@9 00000001400177e0     inftrees.obj
 0002:00001820       ?lext@?1??inflate_table@@9@9 0000000140017820     inftrees.obj
 0002:00001860       ?dbase@?1??inflate_table@@9@9 0000000140017860     inftrees.obj
 0002:000018a0       ?dext@?1??inflate_table@@9@9 00000001400178a0     inftrees.obj
 0002:00001be0       extra_lbits                0000000140017be0     trees.obj
 0002:00001c60       extra_dbits                0000000140017c60     trees.obj
 0002:00001ce0       extra_blbits               0000000140017ce0     trees.obj
 0002:00001d30       bl_order                   0000000140017d30     trees.obj
 0002:00001d50       static_ltree               0000000140017d50     trees.obj
 0002:000021d0       static_dtree               00000001400181d0     trees.obj
 0002:00002250       base_length                0000000140018250     trees.obj
 0002:000022d0       base_dist                  00000001400182d0     trees.obj
 0002:00002348       static_l_desc              0000000140018348     trees.obj
 0002:00002368       static_d_desc              0000000140018368     trees.obj
 0002:00002388       static_bl_desc             0000000140018388     trees.obj
 0002:000023b0       crc_table                  00000001400183b0     zcrc32.obj
 0002:000027b0       crc_big_table              00000001400187b0     zcrc32.obj
 0002:00002bb0       crc_braid_table            0000000140018bb0     zcrc32.obj
 0002:00003bb0       crc_braid_big_table        0000000140019bb0     zcrc32.obj
 0002:00004bb0       x2n_table                  000000014001abb0     zcrc32.obj
 0002:00004d10       ?all_band_inits@@3QBUband_init@@B 000000014001ad10     bands.obj
 0002:00006950       ?ERB@@3QBDB                000000014001c950     coding.obj
 0002:00006a70       ?flag_opts@@3QBDB          000000014001ca70     main.obj
 0002:00006a78       ?string_opts@@3QBDB        000000014001ca78     main.obj
 0002:00006a80       ?sccsver@@3QBDB            000000014001ca80     main.obj
 0002:00007070       ?TAG_ORDER@@3QBCB          000000014001d070     unpack.obj
 0002:00007088       ?str_tf@@3QBDB             000000014001d088     unpack.obj
 0002:00007098       ?TAGS_IN_ORDER@@3QBCB      000000014001d098     unpack.obj
 0002:00007ee8       ?jarmagic@@3QBGB           000000014001dee8     zip.obj
 0002:00007ef0       ?marker_comment@@3QBDB     000000014001def0     zip.obj
 0002:00008098       GS_ExceptionPointers       000000014001e098     MSVCRT:gs_report.obj
 0002:000085f8       $unwind$deflate            000000014001e5f8     deflate.obj
 0002:000085f8       $unwind$deflateInit2_      000000014001e5f8     deflate.obj
 0002:000085f8       $unwind$?hashTabRef@cpool@@QEAAAEAPEAUentry@@CAEAUbytes@@@Z 000000014001e5f8     unpack.obj
 0002:00008614       $unwind$deflateEnd         000000014001e614     deflate.obj
 0002:00008614       $unwind$updatewindow       000000014001e614     inflate.obj
 0002:00008614       $unwind$?getIntTotal@band@@QEAAHXZ 000000014001e614     bands.obj
 0002:00008614       $unwind$?calloc_heap@unpacker@@QEAAPEAX_K0_N1@Z 000000014001e614     unpack.obj
 0002:0000862c       $unwind$deflateReset       000000014001e62c     deflate.obj
 0002:0000862c       $unwind$deflateResetKeep   000000014001e62c     deflate.obj
 0002:0000862c       $unwind$lm_init            000000014001e62c     deflate.obj
 0002:0000862c       $unwind$_tr_stored_block   000000014001e62c     trees.obj
 0002:0000862c       $unwind$?compareTo@bytes@@QEAAHAEAU1@@Z 000000014001e62c     bytes.obj
 0002:0000862c       $unwind$?ensureSize@fillbytes@@QEAAX_K@Z 000000014001e62c     bytes.obj
 0002:0000862c       $unwind$?writeTo@bytes@@QEAAPEACPEAC@Z 000000014001e62c     bytes.obj
 0002:0000862c       $unwind$?findBySpec@coding@@SAPEAU1@H@Z 000000014001e62c     coding.obj
 0002:0000862c       $unwind$?read_magic@@YAHPEAUunpacker@@QEADH@Z 000000014001e62c     main.obj
 0002:0000862c       $unwind$?free@attr_definitions@unpacker@@QEAAXXZ 000000014001e62c     unpack.obj
 0002:0000862c       $unwind$?parseNumeral@attr_definitions@unpacker@@QEAAPEBDPEBDAEAH@Z 000000014001e62c     unpack.obj
 0002:0000862c       $unwind$?put_space@unpacker@@QEAAPEAC_K@Z 000000014001e62c     unpack.obj
 0002:0000862c       $unwind$?put_stackmap_type@unpacker@@QEAAXXZ 000000014001e62c     unpack.obj
 0002:0000862c       $unwind$?putref@unpacker@@QEAAXPEAUentry@@@Z 000000014001e62c     unpack.obj
 0002:0000862c       $unwind$?putu1ref@unpacker@@QEAAXPEAUentry@@@Z 000000014001e62c     unpack.obj
 0002:0000862c       $unwind$?typeSize@entry@@QEAAHXZ 000000014001e62c     unpack.obj
 0002:0000862c       $unwind$?closeJarFile@jar@@QEAAX_N@Z 000000014001e62c     zip.obj
 0002:0000862c       $unwind$?init@gunzip@@QEAAXPEAUunpacker@@@Z 000000014001e62c     zip.obj
 0002:0000862c       $unwind$?init@jar@@QEAAXPEAUunpacker@@@Z 000000014001e62c     zip.obj
 0002:0000862c       $unwind$?openJarFile@jar@@QEAAXPEBD@Z 000000014001e62c     zip.obj
 0002:0000862c       $unwind$_RTC_Initialize    000000014001e62c     MSVCRT:initsect.obj
 0002:0000862c       $unwind$_RTC_Terminate     000000014001e62c     MSVCRT:initsect.obj
 0002:0000862c       $unwind$__scrt_unhandled_exception_filter 000000014001e62c     MSVCRT:utility_desktop.obj
 0002:00008638       $unwind$deflate_stored     000000014001e638     deflate.obj
 0002:00008654       $unwind$deflate_fast       000000014001e654     deflate.obj
 0002:0000866c       $unwind$deflate_rle        000000014001e66c     deflate.obj
 0002:0000866c       $unwind$deflate_slow       000000014001e66c     deflate.obj
 0002:0000866c       $unwind$_tr_flush_block    000000014001e66c     trees.obj
 0002:0000866c       $unwind$send_all_trees     000000014001e66c     trees.obj
 0002:0000866c       $unwind$?read_attr_defs@unpacker@@QEAAXXZ 000000014001e66c     unpack.obj
 0002:00008688       $unwind$deflate_huff       000000014001e688     deflate.obj
 0002:00008688       $unwind$flush_pending      000000014001e688     deflate.obj
 0002:00008688       $unwind$read_buf           000000014001e688     deflate.obj
 0002:00008688       $unwind$inflateReset2      000000014001e688     inflate.obj
 0002:00008688       $unwind$?getRefCommon@band@@QEAAPEAUentry@@PEAUcpindex@@_N@Z 000000014001e688     bands.obj
 0002:00008688       $unwind$?getInt@value_stream@@QEAAHXZ 000000014001e688     coding.obj
 0002:00008688       $unwind$?ensure_input@unpacker@@QEAA_N_J@Z 000000014001e688     unpack.obj
 0002:00008688       $unwind$?free@unpacker@@QEAAXXZ 000000014001e688     unpack.obj
 0002:00008688       $unwind$?readBandData@attr_definitions@unpacker@@QEAAXH@Z 000000014001e688     unpack.obj
 0002:00008688       $unwind$?requestOutputIndex@entry@@QEAAXAEAUcpool@@H@Z 000000014001e688     unpack.obj
 0002:0000869c       $unwind$fill_window        000000014001e69c     deflate.obj
 0002:0000869c       $unwind$inflateEnd         000000014001e69c     inflate.obj
 0002:0000869c       $unwind$inflateInit2_      000000014001e69c     inflate.obj
 0002:0000869c       $unwind$?getLong@band@@QEAA_JAEAU1@_N@Z 000000014001e69c     bands.obj
 0002:0000869c       $unwind$?freeAll@ptrlist@@QEAAXXZ 000000014001e69c     bytes.obj
 0002:0000869c       $unwind$?realloc@bytes@@QEAAX_K@Z 000000014001e69c     bytes.obj
 0002:0000869c       $unwind$?saveFrom@bytes@@QEAAXPEBX_K@Z 000000014001e69c     bytes.obj
 0002:0000869c       $unwind$?usage@@YAXPEAUunpacker@@PEBD_N@Z 000000014001e69c     main.obj
 0002:0000869c       $unwind$?buildBands@attr_definitions@unpacker@@QEAAPEAPEAUband@@PEAUlayout_definition@2@@Z 000000014001e69c     unpack.obj
 0002:0000869c       $unwind$?computeOutputIndexes@cpool@@QEAAXXZ 000000014001e69c     unpack.obj
 0002:0000869c       $unwind$?ensure_put_space@unpacker@@QEAAX_K@Z 000000014001e69c     unpack.obj
 0002:0000869c       $unwind$?finish@unpacker@@QEAAXXZ 000000014001e69c     unpack.obj
 0002:0000869c       $unwind$?put_label@unpacker@@QEAAXHH@Z 000000014001e69c     unpack.obj
 0002:0000869c       $unwind$?putref_index@unpacker@@QEAAHPEAUentry@@H@Z 000000014001e69c     unpack.obj
 0002:0000869c       $unwind$?read_classes@unpacker@@QEAAXXZ 000000014001e69c     unpack.obj
 0002:0000869c       $unwind$?read_files@unpacker@@QEAAXXZ 000000014001e69c     unpack.obj
 0002:0000869c       $unwind$?redirect_stdio@unpacker@@QEAAXXZ 000000014001e69c     unpack.obj
 0002:0000869c       $unwind$?read_fixed_field@gunzip@@QEAAXPEAD_K@Z 000000014001e69c     zip.obj
 0002:000086ac       $unwind$longest_match      000000014001e6ac     deflate.obj
 0002:000086c8       $unwind$inflate_fast       000000014001e6c8     inffast.obj
 0002:000086e0       $unwind$inflate            000000014001e6e0     inflate.obj
 0002:000086f8       $unwind$inflateReset       000000014001e6f8     inflate.obj
 0002:000086f8       $unwind$inflateResetKeep   000000014001e6f8     inflate.obj
 0002:000086f8       $unwind$?abort@attr_definitions@unpacker@@QEAAXPEBD@Z 000000014001e6f8     unpack.obj
 0002:000086f8       $unwind$?abort@cpool@@QEAAXPEBD@Z 000000014001e6f8     unpack.obj
 0002:000086f8       $unwind$?abort@unpacker@@QEAAXPEBD@Z 000000014001e6f8     unpack.obj
 0002:000086f8       $unwind$?getKQIndex@cpool@@QEAAPEAUcpindex@@XZ 000000014001e6f8     unpack.obj
 0002:000086f8       $unwind$?start@unpacker@@QEAAXPEAX_K@Z 000000014001e6f8     unpack.obj
 0002:000086f8       $unwind$?to_bci@unpacker@@QEAAII@Z 000000014001e6f8     unpack.obj
 0002:000086f8       $unwind$?unpack_aborting@@YA_NPEAUunpacker@@@Z 000000014001e6f8     utils.obj
 0002:000086f8       $unwind$__scrt_initialize_default_local_stdio_options 000000014001e6f8     MSVCRT:default_local_stdio_options.obj
 0002:000086f8       $unwind$?post_pgo_initialization@@YAHXZ 000000014001e6f8     MSVCRT:exe_main.obj
 0002:000086f8       $unwind$?pre_cpp_initialization@@YAXXZ 000000014001e6f8     MSVCRT:exe_main.obj
 0002:000086f8       $unwind$mainCRTStartup     000000014001e6f8     MSVCRT:exe_main.obj
 0002:000086f8       $unwind$__report_rangecheckfailure 000000014001e6f8     MSVCRT:gs_report.obj
 0002:000086f8       $unwind$__GSHandlerCheck   000000014001e6f8     MSVCRT:gshandler.obj
 0002:000086f8       $unwind$__scrt_acquire_startup_lock 000000014001e6f8     MSVCRT:utility.obj
 0002:000086f8       $unwind$atexit             000000014001e6f8     MSVCRT:utility.obj
 0002:000086f8       $unwind$__scrt_is_managed_app 000000014001e6f8     MSVCRT:utility_desktop.obj
 0002:00008700       $unwind$inflate_table      000000014001e700     inftrees.obj
 0002:00008724       $unwind$pqdownheap         000000014001e724     trees.obj
 0002:00008730       $unwind$gen_bitlen         000000014001e730     trees.obj
 0002:00008748       $unwind$build_tree         000000014001e748     trees.obj
 0002:00008768       $unwind$scan_tree          000000014001e768     trees.obj
 0002:00008780       $unwind$send_tree          000000014001e780     trees.obj
 0002:0000879c       $unwind$compress_block     000000014001e79c     trees.obj
 0002:000087b4       $unwind$crc32_z            000000014001e7b4     zcrc32.obj
 0002:000087cc       $unwind$?readData@band@@QEAAXH@Z 000000014001e7cc     bands.obj
 0002:000087ec       $unwind$?getIntCount@band@@QEAAHH@Z 000000014001e7ec     bands.obj
 0002:000087ec       $unwind$?makeBands@band@@SAPEAU1@PEAUunpacker@@@Z 000000014001e7ec     bands.obj
 0002:000087ec       $unwind$?get_next_file@unpacker@@QEAAPEAUfile@1@XZ 000000014001e7ec     unpack.obj
 0002:00008804       $unwind$?free@bytes@@QEAAXXZ 000000014001e804     bytes.obj
 0002:00008804       $unwind$?malloc@bytes@@QEAAX_K@Z 000000014001e804     bytes.obj
 0002:00008804       $unwind$?setCoding@value_stream@@QEAAXPEAUcoding@@@Z 000000014001e804     coding.obj
 0002:00008804       $unwind$?nbasename@@YAPEBDPEBD@Z 000000014001e804     main.obj
 0002:00008804       $unwind$?putu2@unpacker@@QEAAXH@Z 000000014001e804     unpack.obj
 0002:00008804       $unwind$?putu4@unpacker@@QEAAXH@Z 000000014001e804     unpack.obj
 0002:00008804       $unwind$?putu8@unpacker@@QEAAX_J@Z 000000014001e804     unpack.obj
 0002:00008804       $unwind$?read_bands@unpacker@@QEAAXXZ 000000014001e804     unpack.obj
 0002:00008804       $unwind$?reset_cur_classfile@unpacker@@QEAAXXZ 000000014001e804     unpack.obj
 0002:00008804       $unwind$?must_calloc@@YAPEAX_K0@Z 000000014001e804     utils.obj
 0002:00008804       $unwind$?unpack_abort@@YAXPEBDPEAUunpacker@@@Z 000000014001e804     utils.obj
 0002:00008804       $unwind$?free@gunzip@@QEAAXXZ 000000014001e804     zip.obj
 0002:00008804       $unwind$?pre_c_initialization@@YAHXZ 000000014001e804     MSVCRT:exe_main.obj
 0002:00008804       $unwind$__raise_securityfailure 000000014001e804     MSVCRT:gs_report.obj
 0002:00008804       $unwind$__scrt_initialize_crt 000000014001e804     MSVCRT:utility.obj
 0002:00008804       $unwind$__scrt_initialize_onexit_tables 000000014001e804     MSVCRT:utility.obj
 0002:00008804       $unwind$__scrt_release_startup_lock 000000014001e804     MSVCRT:utility.obj
 0002:00008804       $unwind$__scrt_uninitialize_crt 000000014001e804     MSVCRT:utility.obj
 0002:00008804       $unwind$_onexit            000000014001e804     MSVCRT:utility.obj
 0002:0000880c       $unwind$?grow@fillbytes@@QEAAPEAC_K@Z 000000014001e80c     bytes.obj
 0002:0000880c       $unwind$?saveTo@unpacker@@QEAAXAEAUbytes@@PEAC_K@Z 000000014001e80c     unpack.obj
 0002:00008820       $unwind$?init@coding@@QEAAPEAU1@XZ 000000014001e820     coding.obj
 0002:00008820       $unwind$?get_code_header@unpacker@@QEAAXAEAH000@Z 000000014001e820     unpack.obj
 0002:00008834       $unwind$?parse@coding@@SAIAEAPEACHH@Z 000000014001e834     coding.obj
 0002:00008834       $unwind$?parse_lgH@coding@@SAIAEAPEACHHH@Z 000000014001e834     coding.obj
 0002:00008844       $unwind$?parseMultiple@coding@@SAXAEAPEACHPEACHH@Z 000000014001e844     coding.obj
 0002:00008844       $unwind$__GSHandlerCheckCommon 000000014001e844     MSVCRT:gshandler.obj
 0002:0000884c       $unwind$?init@coding_method@@QEAAXAEAPEACPEAC0HPEAUcoding@@HPEAUintlist@@@Z 000000014001e84c     coding.obj
 0002:0000886c       $unwind$fprintf            000000014001e86c     main.obj
 0002:0000886c       $unwind$sprintf            000000014001e86c     main.obj
 0002:00008878       $unwind$?run@unpacker@@SAHHPEAPEAD@Z 000000014001e878     main.obj
 0002:0000889c       $unwind$?read_input_via_stdio@@YA_JPEAUunpacker@@PEAX_J2@Z 000000014001e89c     main.obj
 0002:0000889c       $unwind$?write_classfile_head@unpacker@@QEAAXXZ 000000014001e89c     unpack.obj
 0002:0000889c       $unwind$?write_classfile_tail@unpacker@@QEAAXXZ 000000014001e89c     unpack.obj
 0002:000088b4       $unwind$_snprintf          000000014001e8b4     unpack.obj
 0002:000088c4       $unwind$?dump_options@unpacker@@QEAAXXZ 000000014001e8c4     unpack.obj
 0002:000088c4       $unwind$?ensureUtf8@cpool@@QEAAPEAUentry@@AEAUbytes@@@Z 000000014001e8c4     unpack.obj
 0002:000088d8       $unwind$?ensureClass@cpool@@QEAAPEAUentry@@AEAUbytes@@@Z 000000014001e8d8     unpack.obj
 0002:000088ec       $unwind$?init@cpool@@QEAAXPEAUunpacker@@QEAH@Z 000000014001e8ec     unpack.obj
 0002:000088ec       $unwind$?popBody@attr_definitions@unpacker@@QEAAPEAPEAUband@@H@Z 000000014001e8ec     unpack.obj
 0002:000088fc       $unwind$?expandSignatures@cpool@@QEAAXXZ 000000014001e8fc     unpack.obj
 0002:00008914       $unwind$?init@unpacker@@QEAAXP6A_JPEAU1@PEAX_J2@Z@Z 000000014001e914     unpack.obj
 0002:00008914       $unwind$?initGroupIndexes@cpool@@QEAAXXZ 000000014001e914     unpack.obj
 0002:00008920       $unwind$?initMemberIndexes@cpool@@QEAAXXZ 000000014001e920     unpack.obj
 0002:00008938       $unwind$?defineLayout@attr_definitions@unpacker@@QEAAPEAUlayout_definition@2@HPEBD0@Z 000000014001e938     unpack.obj
 0002:00008950       $unwind$?parseLayout@attr_definitions@unpacker@@QEAAPEBDPEBDAEAPEAPEAUband@@H@Z 000000014001e950     unpack.obj
 0002:00008968       $unwind$?parseIntLayout@attr_definitions@unpacker@@QEAAPEBDPEBDAEAPEAUband@@C_N@Z 000000014001e968     unpack.obj
 0002:00008984       $unwind$?readBandData@attr_definitions@unpacker@@QEAAXPEAPEAUband@@I@Z 000000014001e984     unpack.obj
 0002:0000899c       $unwind$?reset@unpacker@@QEAAXXZ 000000014001e99c     unpack.obj
 0002:000089b0       $unwind$?set_option@unpacker@@QEAA_NPEBD0@Z 000000014001e9b0     unpack.obj
 0002:000089c4       $unwind$?get_option@unpacker@@QEAAPEBDPEBD@Z 000000014001e9c4     unpack.obj
 0002:000089dc       $unwind$?read_cp@unpacker@@QEAAXXZ 000000014001e9dc     unpack.obj
 0002:000089dc       $unwind$?write_file_to_jar@unpacker@@QEAAXPEAUfile@1@@Z 000000014001e9dc     unpack.obj
 0002:000089f4       $unwind$?checkLegacy@unpacker@@QEAAXPEBD@Z 000000014001e9f4     unpack.obj
 0002:00008a08       $unwind$?putlayout@unpacker@@QEAAXPEAPEAUband@@@Z 000000014001ea08     unpack.obj
 0002:00008a24       $unwind$?write_code@unpacker@@QEAAXXZ 000000014001ea24     unpack.obj
 0002:00008a34       $unwind$?write_bc_ops@unpacker@@QEAAXXZ 000000014001ea34     unpack.obj
 0002:00008a4c       $unwind$?write_members@unpacker@@QEAAXHH@Z 000000014001ea4c     unpack.obj
 0002:00008a64       $unwind$?write_attrs@unpacker@@QEAAHH_K@Z 000000014001ea64     unpack.obj
 0002:00008a88       $unwind$?write_ics@unpacker@@QEAAHHH@Z 000000014001ea88     unpack.obj
 0002:00008aa4       $unwind$?write_bsms@unpacker@@QEAAHHH@Z 000000014001eaa4     unpack.obj
 0002:00008ac0       $unwind$?read_file_header@unpacker@@QEAAXXZ 000000014001eac0     unpack.obj
 0002:00008ae8       $unwind$?read_ics@unpacker@@QEAAXXZ 000000014001eae8     unpack.obj
 0002:00008b04       $unwind$?read_attrs@unpacker@@QEAAXHH@Z 000000014001eb04     unpack.obj
 0002:00008b1c       $unwind$?read_code_headers@unpacker@@QEAAXXZ 000000014001eb1c     unpack.obj
 0002:00008b1c       $unwind$?start@gunzip@@QEAAXH@Z 000000014001eb1c     zip.obj
 0002:00008b2c       $unwind$?read_bcs@unpacker@@QEAAXXZ 000000014001eb2c     unpack.obj
 0002:00008b44       $unwind$?read_Utf8_values@unpacker@@QEAAXPEAUentry@@HC@Z 000000014001eb44     unpack.obj
 0002:00008b5c       $unwind$?read_single_words@unpacker@@QEAAXAEAUband@@PEAUentry@@HCH@Z 000000014001eb5c     unpack.obj
 0002:00008b78       $unwind$?read_double_words@unpacker@@QEAAXAEAUband@@PEAUentry@@HCH@Z 000000014001eb78     unpack.obj
 0002:00008b90       $unwind$?read_single_refs@unpacker@@QEAAXAEAUband@@CPEAUentry@@HCH@Z 000000014001eb90     unpack.obj
 0002:00008ba8       $unwind$?read_double_refs@unpacker@@QEAAXAEAUband@@CCPEAUentry@@HC@Z 000000014001eba8     unpack.obj
 0002:00008bc0       $unwind$?read_signature_values@unpacker@@QEAAXPEAUentry@@HC@Z 000000014001ebc0     unpack.obj
 0002:00008bdc       $unwind$?read_method_handle@unpacker@@QEAAXPEAUentry@@HCH@Z 000000014001ebdc     unpack.obj
 0002:00008bdc       $unwind$?read_method_type@unpacker@@QEAAXPEAUentry@@HCH@Z 000000014001ebdc     unpack.obj
 0002:00008bf8       $unwind$?read_bootstrap_methods@unpacker@@QEAAXPEAUentry@@HC@Z 000000014001ebf8     unpack.obj
 0002:00008c14       $unwind$?compare_Utf8_chars@@YAHAEAUbytes@@0@Z 000000014001ec14     unpack.obj
 0002:00008c2c       $unwind$?addJarEntry@jar@@QEAAXPEBD_NHAEAUbytes@@2@Z 000000014001ec2c     zip.obj
 0002:00008c44       $unwind$?write_data@jar@@QEAAXPEAX_K@Z 000000014001ec44     zip.obj
 0002:00008c54       $unwind$?add_to_jar_directory@jar@@QEAAXPEBD_NHHHK@Z 000000014001ec54     zip.obj
 0002:00008c74       $unwind$?write_jar_header@jar@@QEAAXPEBD_NHHHI@Z 000000014001ec74     zip.obj
 0002:00008c90       $unwind$?write_jar_extra@jar@@QEAAXHHI@Z 000000014001ec90     zip.obj
 0002:00008ca0       $unwind$?write_central_directory@jar@@QEAAXXZ 000000014001eca0     zip.obj
 0002:00008cc4       $unwind$?dostime@jar@@QEAAKHHHHHH@Z 000000014001ecc4     zip.obj
 0002:00008ccc       $unwind$?get_dostime@jar@@QEAAKH@Z 000000014001eccc     zip.obj
 0002:00008ce0       $unwind$?deflate_bytes@jar@@QEAA_NAEAUbytes@@0@Z 000000014001ece0     zip.obj
 0002:00008cfc       $unwind$?read_input_via_gzip@@YA_JPEAUunpacker@@PEAX_J2@Z 000000014001ecfc     zip.obj
 0002:00008d14       $unwind$__report_securityfailure 000000014001ed14     MSVCRT:gs_report.obj
 0002:00008d1c       $unwind$__report_gsfailure 000000014001ed1c     MSVCRT:gs_report.obj
 0002:00008d24       $unwind$capture_current_context 000000014001ed24     MSVCRT:gs_report.obj
 0002:00008d30       $unwind$capture_previous_context 000000014001ed30     MSVCRT:gs_report.obj
 0002:00008d40       $xdatasym                  000000014001ed40     MSVCRT:amdsecgs.obj
 0002:00008d48       $xdatasym                  000000014001ed48     MSVCRT:chkstk.obj
 0002:00008d50       $unwind$?__scrt_common_main_seh@@YAHXZ 000000014001ed50     MSVCRT:exe_main.obj
 0002:00008d88       $unwind$?filt$0@?0??__scrt_common_main_seh@@YAHXZ@4HA 000000014001ed88     MSVCRT:exe_main.obj
 0002:00008d90       $unwind$__scrt_is_nonwritable_in_current_image 000000014001ed90     MSVCRT:utility.obj
 0002:00008db0       $unwind$__scrt_is_nonwritable_in_current_image$filt$0 000000014001edb0     MSVCRT:utility.obj
 0002:00008db8       $unwind$__security_init_cookie 000000014001edb8     MSVCRT:gs_support.obj
 0002:00008dc4       $unwind$__scrt_fastfail    000000014001edc4     MSVCRT:utility_desktop.obj
 0002:00008dd4       $unwind$__isa_available_init 000000014001edd4     MSVCRT:cpu_disp.obj
 0002:00008de8       $xdatasym                  000000014001ede8     MSVCRT:guard_dispatch.obj
 0002:00008df0       $xdatasym                  000000014001edf0     MSVCRT:guard_xfg_dispatch.obj
 0002:00008e00       .edata                     000000014001ee00     unpack200.exp
 0002:00008e28       rgpv                       000000014001ee28     unpack200.exp
 0002:00008e2c       rgszName                   000000014001ee2c     unpack200.exp
 0002:00008e30       rgwOrd                     000000014001ee30     unpack200.exp
 0002:00008e32       szName                     000000014001ee32     unpack200.exp
 0002:00008e40       $N00001                    000000014001ee40     unpack200.exp
 0002:0000937e       .idata$6                   000000014001f37e     kernel32:KERNEL32.dll
 0002:0000940a       .idata$6                   000000014001f40a     vcruntime:VCRUNTIME140.dll
 0002:0000970c       .idata$6                   000000014001f70c     ucrt:api-ms-win-crt-heap-l1-1-0.dll
 0002:0000972c       .idata$6                   000000014001f72c     ucrt:api-ms-win-crt-stdio-l1-1-0.dll
 0002:0000974c       .idata$6                   000000014001f74c     ucrt:api-ms-win-crt-filesystem-l1-1-0.dll
 0002:00009772       .idata$6                   000000014001f772     ucrt:api-ms-win-crt-runtime-l1-1-0.dll
 0002:00009794       .idata$6                   000000014001f794     ucrt:api-ms-win-crt-string-l1-1-0.dll
 0002:000097b6       .idata$6                   000000014001f7b6     ucrt:api-ms-win-crt-environment-l1-1-0.dll
 0002:000097dc       .idata$6                   000000014001f7dc     ucrt:api-ms-win-crt-utility-l1-1-0.dll
 0002:000097fe       .idata$6                   000000014001f7fe     ucrt:api-ms-win-crt-convert-l1-1-0.dll
 0002:00009820       .idata$6                   000000014001f820     ucrt:api-ms-win-crt-time-l1-1-0.dll
 0002:00009840       .idata$6                   000000014001f840     ucrt:api-ms-win-crt-math-l1-1-0.dll
 0002:00009860       .idata$6                   000000014001f860     ucrt:api-ms-win-crt-locale-l1-1-0.dll
 0003:00000b00       ?keys@?M@??next_arg@@YAHAEAPEAPEAD@Z@4PAPEBDA 0000000140020b00     main.obj
 0003:00000b40       ?opts@?1??dump_options@unpacker@@QEAAXXZ@4PAPEBDA 0000000140020b40     unpack.obj
 0003:00000bb0       ?dummy@@3PACA              0000000140020bb0     bytes.obj
 0003:00000fb0       ?no_meta@@3PAPEBCA         0000000140020fb0     coding.obj
 0003:00000fc0       ?suppress_warning@@3_NA    0000000140020fc0     main.obj
 0003:00000fd0       ?no_bands@@3PAPEAUband@@A  0000000140020fd0     unpack.obj
 0003:00000fe0       GS_ExceptionRecord         0000000140020fe0     MSVCRT:gs_report.obj
 0003:00001080       GS_ContextRecord           0000000140021080     MSVCRT:gs_report.obj
 0003:00001560       ?is_initialized_as_dll@@3_NA 0000000140021560     MSVCRT:utility.obj
 0003:00001561       ?module_local_atexit_table_initialized@@3_NA 0000000140021561     MSVCRT:utility.obj
 0003:00001568       ?module_local_atexit_table@@3U_onexit_table_t@@A 0000000140021568     MSVCRT:utility.obj
 0003:00001580       ?module_local_at_quick_exit_table@@3U_onexit_table_t@@A 0000000140021580     MSVCRT:utility.obj
 0005:00000060       $R000000                   0000000140023060     unpack200.exe.res
